:020000000C945E
:1000020070000C9400000C9400000C9400000C94FE
:1000120000000C9400000C9400000C9400000C945E
:1000220000000C9400000C9400000C9400000C944E
:1000320000000C9400000C9400000C9400000C943E
:10004200D2000C9400000C949F000C9400000C94BD
:1000520000000C9400000C9400000C9400000C941E
:1000620000000C9400001027E80364000A0001005D
:100072000010000110000100000000000A00000052
:10008200000000000000000000000000000000006E
:10009200000000000000000000000000000000005E
:1000A200000000000000000000000000000000004E
:1000B2000000000000000000000A0A0A0A0A0A0AF8
:1000C2000A0A0A0A0A0A0A0A0A00020002007A0056
:1000D200020004007C00010007037E000000F89487
:1000E200EE27EFBBF1E0F5BFE5BF8DE0A2E0BB2755
:1000F200ED938A95E9F780E098E0A0E0B1E0ED9316
:100102000197E9F7ECECF0E085919591009761F0A9
:10011200A591B59105901590BF01F00105900D9242
:100122000197E1F7FB01F0CFE8E0EEBBEFEFEDBFA7
:10013200E8E0EEBFC0E0D3E00C94C903AA93EA93CF
:10014200FA93EFB7EA931A930A931091C0000091C1
:10015200C600E12FEC71E9F4E0910D04EF5FE0934A
:100162000D04E150F0E0EC50FC4F0083A0910D042F
:10017200A93119F4E0E0E0930D04A0910F04AF5F00
:10018200A0930F04A93129F4E0E0E0930F046894EE
:1001920037F809911991E991EFBFF991E991A99184
:1001A20018950A921A926A937A938A939A93AA93C7
:1001B200BA93EA93FA93EFB7EA93E0914A03F09184
:1001C2004B033196E0934A03F0934B030E94FC29C0
:1001D200E1E5F1E00E943F360E2E0E94FC29E3EA9F
:1001E200F2E00E943F36E02909F40BC2A0914803D5
:1001F200B0914903E5E0F0E00E9463360E2EA09133
:100202002703EEE00E943536E02121F0E09127033A
:10021200EF5F03C025FC03C0E0E0E0932703A09159
:100222002703AE3011F4689425F8A0913003A13071
:1002320029F4F79B02C0F79801C0F79AE1E02E2655
:100242000E94012A0E940A2AE093D803F093D9035C
:100252006093DA037093DB030E94112AACEBB3E0E4
:100262000E94162A0E941D2AA8EEB3E00E94162AB6
:100272000E94222A0E942B2A0E946635E093BC0328
:10028200F093BD036093BE037093BF03A091E80394
:10029200B091E9038091EA039091EB03E0E0F0E092
:1002A20060E772E40E946635E093E803F093E903A5
:1002B2006093EA037093EB030E94302A0E94352A6E
:1002C2000E2E0E943A2A0E94352AE02161F1E09125
:1002D200E803F091E9036091EA037091EB030E9455
:1002E200222A0E946635E093E403F093E5036093CB
:1002F200E6037093E7030E943F2AACE5B3E00E9455
:10030200482AA091E403B091E5038091E60390911D
:10031200E7030E940A2AE093C403F093C5036093A3
:10032200C6037093C7030E944D2A0E945E2A0E9450
:10033200C834E093CC03F093CD036093CE03709363
:10034200CF030E944D2A0E94672A0E94C834E0937C
:10035200F003F093F1036093F2037093F3030E94AE
:10036200702A0E94792A0E948C2AA4EAB3E00E9491
:1003720057340E944D370E94702AAAE0B0E080E014
:1003820090E00E9491360E94672A0E948C340E945B
:10039200AB3570F0E0E0E093F003E093F103E0931B
:1003A200F203E093F3030E94912A31960E94962A67
:1003B200E091A803F091A9036091AA037091AB03A5
:1003C200A091D003B091D1038091D2039091D30335
:1003D2000E941835DF01CB010E940A2AE093DC0358
:1003E200F093DD036093DE037093DF030E949B2A88
:1003F2000E94C8340E94A42AE0910E03F0E00E94F9
:10040200AD2A0E940D360E94B62AACE7B3E00E94E4
:10041200C52A0E94012A0E94AD373CF5A091DC0357
:10042200B091DD038091DE039091DF030E94CA2A1E
:100432007F936F93FF93EF93A091D803B091D90369
:100442008091DA039091DB030E94CA2AAF91BF9197
:100452008F919F910E946635E093D403F093D50368
:100462006093D6037093D70309C0E0E0E093D4030E
:10047200E093D503E093D603E093D703A091D7038B
:10048200AA238AF40E94D12A0E94DA2A18F40E942E
:10049200E12A08C00E94E82A0E942234A4E8B3E0BC
:1004A2000E94C52A14C00E94D12AE0E0F0EC69E75C
:1004B20074E40E94AB3509F008F403C00E94E12AFB
:1004C20006C00E94E82AA4E8B3E00E94C52A0E945E
:1004D200F12A0E94FA2A0E94C8340E94032BE0915A
:1004E200BC03F091BD036091BE037091BF030E94F3
:1004F2000C2B0E94AB3568F5E091C403F091C50363
:100502006091C6037091C7030E940C2B0E94C834ED
:10051200E093C003F093C1036093C2037093C303DB
:100522000E940C2B0E94152B0E94C134DF01CB01CB
:100532000E943F2A0E946635A0E0B0E081E695E481
:100542000E941835A8E7B3E00E94C52A689424F8EF
:1005520002C0E0E12E260E94F12A0E941E2B0E9478
:10056200C834E093C803F093C9036093CA0370933D
:10057200CB030E941E2BE0E0F0E060E87FE30E94E4
:10058200AB3509F008F412C0E093C803E093C90345
:10059200E093CA03E093CB030E94272BEF5FFF4F48
:1005A2006F4F7F4F0E94302B0E94392B0E943F2BAE
:1005B200A034E2E4BE07EFE08E07E0E09E0778F0A9
:1005C200E0E0E0936A03E0936B03E0936C03E09353
:1005D2006D03AAE4B0E00E94482B0E9482370E9479
:1005E200FA2A0E944D2BACE4B3E00E94482AA09163
:1005F2002503AC3308F4F298A0912503AC3309F437
:10060200F29A0E94FC29A33AE2E0BE0709F097C0E1
:10061200A09124030E94512B0E94562B0E94482B2A
:100622000E9469360E945F2BE02191F0E091250340
:10063200EF5FE0932503E0912403F0E03296A0916E
:100642002503B0E0EA17FB0719F4ECE3E093250376
:10065200E0E0E0934A03E0934B03D394A0910F03AD
:10066200A13028F4E0910F03EF5FE0930F030E94A3
:10067200662BE8E5F2E00E945D360E2E0E946B2B9F
:10068200E021E9F0E0916003F09161033196E0939B
:100692006003F09361030E94662B0E94702BEA1B99
:1006A200FB0BE0936603F09367030E94562B0E94B4
:1006B200AD372CF4E0E0E0936003E0936103ECE3F8
:1006C200ED1589F4DD24C394EC1569F4CC24E09192
:1006D2000003EF5FE0930003A0910003A43119F43B
:1006E200E0E0E0930003A0912C03A130D0F0E09170
:1006F2001203EF5FE0931203A0911203A23088F07D
:10070200E0911103EF5FE0931103E0E0E093120345
:10071200E0912C03A0911103EA1718F4E0E0E093B2
:100722001103E0912C03E03019F4E0E0E0931103AF
:10073200A0912C03A23019F4E1E0E0931103E991B6
:10074200EFBFF991E991B991A99199918991799123
:100752006991199009901895AA93E881E066E0934F
:100762007C0085E28A95F1F7E0917A00E064E093FB
:100772007A00E0917A00E071E1F3E0917A00E061C1
:10078200E0937A00E0917800F09179002196089543
:10079200EF9762978BE4A6E0B0E0E0E8F0E00E9419
:1007A200C237FF2401E021E0E0E8E0936100E0E0ED
:1007B200E0936100EFE0E4B9E1E0E5B9E0E0E7B938
:1007C200E4E0E8B9EAEFEAB9E7EEEBB9E0E0E4BD6C
:1007D200E3E0E5BDE0E0E6BDE7BDE8BDE093800013
:1007E200E0938100E0938500E0938400E09387002A
:1007F200E0938600E0938900E0938800E0938B0009
:10080200E0938A00E093B600E1EAE093B000E2E010
:10081200E093B100E0E0E093B200E093B300E09334
:10082200B400E1E0E0936E00E0E0E0936F00E0935B
:100832007000E0936900EDBBE0936800E093C000B4
:10084200E8E9E093C100E6E0E093C200E0E0E09373
:10085200C500E7E4E093C400E0E8E0BFE0E0E09335
:100862007F00E0937E00E0E6E0937C00E6E2E09326
:100872007A00E0E0E0937B00ECBDE093BC0078946A
:100882005F9A0E94752B0E94792B0E947F2B0E94F7
:10089200862B0E94932B0E94752BEAE06E1668F459
:1008A200A4E3B0E00E94A02BA7E2B0E0E0E00E9447
:1008B2009237A8E2B0E00E949237EAE09E1650F426
:1008C200AAE3B0E00E94A02BA2E4B0E00E94A02B19
:1008D200689426F8EAE0BE1618F4689430F827F80F
:1008E200689433F8E8E1E09314030E94A52B0E9478
:1008F200AC2B0E94B32BE8ECF0E0E0937203F09390
:100902007303A0E0B0E00E947637E0931503A1E004
:10091200B0E00E947637E0931603A2E0B0E00E94B6
:100922007637E0931703A3E0B0E00E947637E093B6
:100932001903A4E0B0E00E947637E8A7A5E0B0E092
:100942000E947637E9A7A6E0B0E00E947637EAA7D0
:10095200A7E0B0E00E947637E0931A03A8E0B0E087
:100962000E947637E0931B03F798F198AAE0B0E073
:100972000E947637E0932403A2E3B0E00E9472372C
:100982000E94BA2BA3E1B0E00E947637ECA3A4E167
:10099200B0E00E947637EDA3A5E1B0E00E94763781
:1009A200EEA3ABE0B0E00E947637E8A3ACE0B0E0A3
:1009B2000E947637E9A3ADE0B0E00E947637EAA361
:1009C200A6E3B0E00E947237E98BFA8BAEE0B0E0AA
:1009D2000E947637E0933103AFE0B0E00E947637B1
:1009E200E0933303A0E1B0E00E947637E093320354
:1009F200AAE4B0E00E946E370E94302BA4E3B0E07C
:100A02000E947237A8EBB3E00E94BF2B0E94152B05
:100A1200ACE4B3E00E94482A0E94FA2A0E942B2AE0
:100A22000E9466350E94032BA1E1B0E00E94763756
:100A32003E2FA8E3B0E00E947237ED8BFE8BA2E15D
:100A4200B0E00E947637EBA7A8E4B0E00E947237CC
:100A5200EB87FC87AAE3B0E00E947237ACECB3E00C
:100A62000E94BF2BA2E4B0E00E947237ACEEB3E06A
:100A72000E94BF2B0E949B2A0E942B2A0E9466354D
:100A82000E94A42AACE3B0E00E9472370E94C62BF7
:100A9200A0E4B0E00E9472370E940D360E94CB2B78
:100AA200A6E1B0E00E9476370E94BD3723F8AEE39C
:100AB200B0E00E9472370E94D42BA7E1B0E00E94FE
:100AC2007637E0930603A8E1B0E00E947637E09320
:100AD2000803A9E1B0E00E947637E0930903AAE196
:100AE200B0E00E947637E0930A03ABE1B0E00E94E7
:100AF2007637E0930B03ACE1B0E00E947637E093E7
:100B02000C03ADE1B0E00E947637E0932803AEE13A
:100B1200B0E00E947637E0932903AFE1B0E00E9493
:100B22007637E0932A03A0E2B0E00E947637E093A2
:100B32002B03A1E2B0E00E947637E0932C03A2E2FD
:100B4200B0E00E947637E0932D03A3E2B0E00E946A
:100B52007637E0932E03A4E2B0E00E947637E0936A
:100B62002F03A4E4B0E00E9472370E94962AA5E205
:100B7200B0E00E947637E0930E03A6E2B0E00E9456
:100B820076370E94BD3736F8A9E2B0E00E94763788
:100B9200E0931003AAE2B0E00E947637EB8FA6E45E
:100BA200B0E00E947237ED87FE87ABE2B0E00E94B0
:100BB2007637E0933C03ACE2B0E00E947637E093F4
:100BC2003D03ADE2B0E00E947637E0933E03AEE231
:100BD200B0E00E947637E0931C03AFE2B0E00E94DF
:100BE2007637E0931E03A9E0B0E00E947637E093E7
:100BF2001F03A0E3B0E00E947637E0932003A1E355
:100C0200B0E00E947637E093210336FE0BC0A7E2E4
:100C1200B0E00E947637CE2EA8E2B0E00E9476378E
:100C2200E0930003A0910203AE3128F4E0910203A5
:100C3200EF5FE0930203A0910203AE31A1F4E0E082
:100C4200E0933603E0938803E0938903EBE0F0E05E
:100C52000E94D92BE8EBE0933703E0E0E0930D0428
:100C6200E4E1E0930203EB8DE030C1F5A091F403DF
:100C7200ECE30E9417360E2EA091F503E7E00E94E6
:100C820017360E22A0910D04EBE00E941736E021E8
:100C9200C1F0E091F603E0933503E091F703E093AE
:100CA2003603E091F803F0E00E94DE2BE091F903B5
:100CB200F0E00E94D92BE091FA03E09337030E94FF
:100CC200E32BA0910D04AC3048F00E94E92B0E9466
:100CD200A52B0E94F52BE0E0E0930D04AB8DA33031
:100CE20009F070C0A091F403ECE60E9417360E2EB4
:100CF200A091F503EBE00E9417360E22A0910D049D
:100D0200EFE00E941736E02109F446C0E091F703B4
:100D1200E0933503E091F803E0933603E091F903A1
:100D2200F0E00E94DE2BF0918803E0E00E94DE2BCF
:100D3200E091FA03F0E0A0918803B0918903EA0FF1
:100D4200FB1F0E94DE2BA0918803B09189030E94B1
:100D5200FF2B0E94DE2BE091FB03E0934303E09123
:100D6200FE03E0934203E091FF03F0E00E94D92BDF
:100D7200E0910004E0933703E091FC03F0E0E0939C
:100D82008A03F0938B03E091FD03F0E0E0938C0380
:100D9200F0938D030E94E32BA0910D04A03190F0FB
:100DA2000E94E92BE0E0E093F903E093FA030E944A
:100DB200F52BEBE0E093FF03E8EBE0930004E0E0C7
:100DC200E0930D04E8EC5E1630F45394E4E1E5158B
:100DD20011F4E1E04E2E0E94042CE7EAE0937A003F
:100DE200A6E00E94082CEF83F887E7E2E0937A00FE
:100DF2000E94042C0E94792B0E9402360E94FE352A
:100E0200E987FA87E7E2E0937A000E94042C0E94C5
:100E12000F2C3B97A0F1A0E00E94082C66277727B1
:100E22000E94182CA8EEB3E080E090E00E94BC364D
:100E3200DF01CB010E94212C662777270E94FE3614
:100E42000E94182CA8EAB3E00E948E340E944D370B
:100E5200E0910703EF5FE0930703E0910603A0919F
:100E62000703AE1750F00E94262CE093A003F093E4
:100E7200A1036093A2037093A303E894F3F80E9482
:100E82002F2C0E94792B0E947F2B0E94362CA2E0ED
:100E92000E94082CDF01E5E0F0E00E94C1368E2EB0
:100EA2000E942F2C0E94932B8AE48A95F1F70E94CC
:100EB200862B0E94362C0E943D2C0E942F2CE7EAA2
:100EC200E0937A00A5E048DCEF2FF0E01E2F0E94AD
:100ED2002F2C0E940F2CAE2E0E942F2CE09110037B
:100EE200E03009F091C0E1E0E51589F50E94472C58
:100EF2005E9710F4E1E0EE8F0E94472CE2E3F0E00F
:100F02000E9463360E2E0E94472CEAEFF0E00E9408
:100F12005D36E02111F0E2E0EE8F0E94472CAB3FFC
:100F2200E0E0BE0710F0E3E0EE8F1E3110F4E1E0E6
:100F3200ED8F0E944C2CA12FEAEF0E943536E02162
:100F420011F0E2E0ED8F1B3F10F0E3E0ED8F0E9425
:100F5200472CEEE1F0E00E945D360E94522C11F027
:100F6200E4E00AC00E94472CEAEFF0E00E946336F8
:100F72000E94522C11F0E5E0EE8FA12FEEE10E94CB
:100F820035360E945E2C11F0E4E008C0A12FEAEF92
:100F92000E943A360E945E2C11F0E5E0ED8FAE8D94
:100FA2000E94512BAE8D0E946A2C49F0E12F0E94C3
:100FB2006F2C18E2AE81AC3511F40E94752CAE8D07
:100FC2000E947B2CAE8DE5E00E941736E02911F0DD
:100FD2000E94752CAD8D0E94512BAD8D0E946A2C02
:100FE20051F018E2AE8D0E94512BAE8D0E946A2CF8
:100FF20011F00E94752CAD8D0E947B2C0E94802CDA
:10100200E02909F01CE303C0E0E0EE8FED8F0E94BF
:10101200852C0E948B2C0E943536E021E1F0E4E120
:10102200E98F6894F3F8013021F4F398F49A02E01E
:1010320012C0023059F4F498F59AAAA5A13010F022
:1010420003E003C0F598F39A01E005C0033019F4F8
:10105200F598F39A01E00E94472CD39708F453C005
:101062000E94952C0E949A2CE02F0E94A12C10F035
:101072000E94B42CE02F0E94BB2C0E94CF2CAC917A
:10108200A13008F43FC00E94D62C0E94DF2C0E949F
:10109200B8374CF40E94CF2C0E94EB2C0E94D7351B
:1010A2000E94F52C23C00E94FE2C0E94002DEF937B
:1010B2000E94FE2C0E94092DAF91EA2379F00E9432
:1010C200CF2C0E94EB2C0E94DC35A0939003B093AE
:1010D2009103809392039093930308C00E94FE2C85
:1010E2000E94122D1CF00E941C2D0CC0A091900396
:1010F200B091910380919203909193030E942B2DC2
:101102000E94302D04C00E94752C0E941C2D0E944A
:10111200372D0E943D2D0E220E94422D01F10E9488
:10112200472C0E94A93710F4E4E1EF8BA09126032B
:101132000E94512B0E944A2DE02141F0E3E0E0930E
:101142003403E0E0E09326030E94502DE091440333
:10115200E09326036894F0F821F8E894F4F8A0915B
:101162002E03A13069F50E94562D0E2EA091260362
:10117200E8EC0E9435360E94582D39F0F4FE05C085
:10118200E0912603EF5FE0932603A12FE3E30E94A1
:101192003A360E2EE0E50E9435360E22A091260345
:1011A200E0E00E943A360E94582D51F0E091260369
:1011B200E150E093260325FE03C0E3E00E94612D87
:1011C2000E944A2D0E2EA12F0E94642DA09126036B
:1011D2000E94692D21F0E0E0E093270306C0A09170
:1011E2002703A23010F4E89425F8A0912603A13039
:1011F20020F0E0912603F0E002C00E94952CE093DB
:101202004803F09349030E94952C309729F4E894FF
:1012120021F86894F4F816C0A0E021FCA1E00E9435
:101222006E2D0E94562D0E22A0912E030E94692D32
:1012320049F0E0E0E09326030E94752CE89422F83E
:10124200689421F8E09104030E94472CF0E0EA1729
:10125200FB0720F4E0914403E09304030E94732D02
:101262000E9481360E22A09131030E94692D1E2E0A
:101272000E94732D0E9479360E22A09132030E94A1
:10128200692DE12979F0E0914403E0930403A0E0A1
:1012920025FCA1E00E94822D0E94872D19F0E2E038
:1012A2000E94612DA0912603A13078F0689422F863
:1012B2000E94952CA0912603B0E0AE17BF0720F044
:1012C200E09126030E946F2C02C0E89422F80E944B
:1012D2008B2D0E22A0E031FCA1E00E94692D31F09D
:1012E200689431F80E94952C0E94A12D0E948B2DAA
:1012F200E02161F10E94A62D0E94AE2DA4F0A091E2
:101302009C03B0919D03E989FA89EA1BFB0BA3E0D8
:10131200B0E00E94B7360E94B62DAE1BBF0BA09361
:101322007403B09375030E94A62D0E94AD372CF46E
:101332000E94BB2D32970E94A12DA0917503AA2372
:101342002AF4E0E0E0937403E09375030E94C02D59
:101352000E94B33774F50E94C02D0E94DC350E94B2
:10136200AE2D74F0A989BA89E0919C03F0919D0396
:10137200EA1BFB0B0E94B62DEA0FFB1F0E94A12D58
:101382000E94C02D0E94DC35A230E0E0BE07E0E002
:101392008E07E0E09E072CF00E94BB2D31960E9442
:1013A200A12D0E94B62DA93CE0E0BE0714F00E94D8
:1013B200AC2B0E94BB2D0E94472CAE17BF0710F426
:1013C200E89431F80E94BB2D0E94472CEA17FB07D4
:1013D20020F40E94BB2D0E94CD2D0E94D22D0E948E
:1013E200D1350E2EA0E032FCA1E00E94692D41F021
:1013F200689432F80E94E12DE0937603F09377032C
:101402000E94D22D0E94AB3509F008F435C00E942B
:10141200E62DDF01CB01E0E0F0E060E070E40E9445
:10142200AB3509F008F410C00E94E62DA0E0B0E050
:1014320080E890E40E9418350E94F52D0E94FA2D52
:10144200A6E7B3E00E94C52A0E94E62D0E94A337B8
:1014520054F4EBA5F0E00E94F52DAE1BBF0BA09358
:101462007603B0937703A0917703AA232AF4E0E0EE
:10147200E0937603E09377030E94D22D0E94AB356E
:10148200A8F50E94FF2DDF01CB01E0E0F0E060E46F
:1014920070E40E94AB3509F008F414C00E94FF2DDD
:1014A200A0E0B0E080EA90E40E941835DF01CB01B1
:1014B2000E940A2E0E940F2E0E94C834A6E7B3E0B3
:1014C2000E94C52A0E94FF2D0E94A3373CF40E946D
:1014D2000A2E3596E0937603F09377030E94F52D5A
:1014E200A13DE7E0BE0714F00E94B32B0E94E12D5C
:1014F200DF010E940A2EAE17BF0710F4E89432F8FB
:101502000E94E12DDF010E940A2EEA17FB0730F448
:101512000E94F52D0E94FF2B0E94CD2D0E94142EB9
:101522000E9481360E2EA0E034FCA1E00E94692DBB
:1015320031F0689434F80E94E12D0E941B2E0E9423
:10154200142E0E94B3375CF50E94202E0E94AE2D0D
:101552009CF0E0911603F0E0A0919803B0919903FA
:10156200AE1BBF0BE3E0F0E00E94292EAE1BBF0BC7
:10157200A0937E03B0937F030E94202E0E94AD377A
:101582002CF40E94302E32970E941B2EA0917F03D2
:10159200AA232AF4E0E0E0937E03E0937F030E9413
:1015A200142E0E94B8378CF50E94352EA430E0E04C
:1015B200BE07E0E08E07E0E09E078CF0A0911603E4
:1015C200BB27E0919803F0919903AE1BBF0BE2E0B9
:1015D200F0E00E94292EEA0FFB1F0E941B2E0E94A0
:1015E200352E0E94AD372CF40E94302E32960E9486
:1015F2001B2EA0917E03B0917F03A13DE7E0BE07C1
:1016020024F0E0EDF7E00E941B2E0E94E12DDF01A5
:101612000E94302EAE17BF0710F4E89434F80E94EF
:10162200E12DDF010E94302EEA17FB0740F4A09162
:101632007E03B0917F030E94FF2B0E94CD2DE0918B
:1016420013030E94472CF0E0EA17FB0720F4E09115
:101652004403E0931303E0911303F0E035970E94F3
:10166200472C0E945D366E2F0E2EA0E031FCA1E0C9
:101672000E94452E1E2E062EA0E032FCA1E00E9402
:10168200452E1E2A062EA0E034FCA1E00E94452E23
:10169200E12949F0E0914403E093130325FE03C0DE
:1016A200E2E00E94612DA0913403A13078F00E9403
:1016B200752CA0913403A13021F4EAE0F0E00E94FD
:1016C200CD2DE0913403E150E09334030E944C2C81
:1016D200A0912E030E94692D1E2EA12FE0E50E94EB
:1016E2003A360E2EA0912E03E1E00E9417360E9498
:1016F200582D1E2A0E944C2CA0912E03E1E00E943C
:1017020017360E220E94872DE129E1F0E0E0E093F6
:101712000503A0912603A13018F0E2E0E093340320
:10172200E0E0E0932603E12FF0E0F2970E940F2E13
:10173200A6EFB8E28CE99FE30E9418350E94553467
:101742001E2F01C010E00E94952CEF87F88BA12F6D
:101752000E94512BA09129030E94452E11F0299A33
:1017620001C02998A12F0E94512BA0913C03E2E0D5
:101772000E941736E02111F0EFEF01C0E0E0E093A4
:101782003F03A82DE4E60E9435366E2F0E2E0E94EE
:101792004A2E0E22AE81EDE50E941C360E94512E89
:1017A2001E2E062E0E944A2E0E220E943D2DE02160
:1017B2001E2A0E94702B0E94662B0E943F360E94B6
:1017C200582E0E946B2BE021E12931F1E0914C036C
:1017D200F0914D03A4E3B0E00E94602E0E94662EB9
:1017E2000E949B2A0E944D2B0E94732E0E94782EEB
:1017F200EC2DA7E2B0E00E947C2EE0910003A8E26B
:10180200B0E00E9492370E94752B5F98A8EEB3E079
:101812000E9418345F98FECFAB2D0E94822E0E9448
:101822003D2DE02131F0E894F2F827F8E0E0E09372
:101832003B030E94872E0E943D2DE02171F0E09132
:101842003B03EF5FE0933B03A0913B03AA3029F4F3
:10185200E0E0E0933B03E09330030E94872EA0E098
:10186200F2FCA1E00E94642D0E943D2DE021B9F11D
:10187200E4E1E88F6894F2F8E0913003EF5FE093DF
:1018820030030E94902E0E94422D19F0E1E0E09375
:101892003003A09130030E947B2C0E94422D19F04C
:1018A200E2E0E09330030E94902EA09129030E946F
:1018B200642DAB8DE3E00E941C36E02119F0E1E0DB
:1018C200E0933003A09130030E947B2CA0E0F0FC57
:1018D200A1E00E94452E19F0E3E0E0933003E0918D
:1018E2003003E03031F4F7982A98E0E0E0934003C7
:1018F2001EC0A0913003A13031F42A98EFEFE0939B
:101902004003E0E014C0A0913003A23039F4F79A0A
:101912002A98EFEFE0934003E0E009C0A091300382
:10192200A33039F4F79A2A9AEFEFE0934003E09359
:1019320041030E94972EE081E093B4000E94562D4D
:101942000E2EA12FE0E00E943A360E220E94872D31
:1019520029F1A0912803A13009F45C9AE0910303D4
:10196200EF5FE0930303A0910303E5E00E943A36A0
:101972000E2EE4E10E943536E02141F0E0910303AE
:10198200E170AFEFEA02F001E093B400A09103032B
:10199200A03118F0E0E0E093030325C05C98A0E0DA
:1019A20030FCA1E00E94822DA09130030E94692D9B
:1019B200D1F0E0913A03EF5FE0933A03A0913A034A
:1019C200A13019F4EFEFE093B400A0913A03A330F1
:1019D20019F4E0E0E093B400A0913A03A43019F4C2
:1019E200E0E0E0933A030E949D2E0E94A42EE1F0D3
:1019F200E0911B03A0911D03AE1728F4E0911D0393
:101A0200EE5FE0931D03E0911B03A0911D03EA1713
:101A120028F4E0911D03E250E0931D03233621F4E4
:101A2200E0911B03E0931D030E949D2EEA17FB0722
:101A3200E0F4E0911C03A0911D03AE1728F4E0919D
:101A42001D03EE5FE0931D03E0911C03A0911D03B3
:101A5200EA1728F4E0911D03E250E0931D032336B8
:101A620021F4E0911C03E0931D03E0911D03E09338
:101A7200B300EAE0E91518F4E894F1F826F80E94B8
:101A8200AD2EA0E026FCA1E00E94642DA0E0F1FCB6
:101A9200A1E00E94642D0E943D2DE02139F168945D
:101AA200F1F8E0910D03EF5FE0930D03E0E0EC8FBE
:101AB200AC8DA53088F40E94B32EA081A13018F01D
:101AC200E5E0EC8F05C0E0910D03EF5FE0930D03BD
:101AD200EC8DEF5FEC8FECCFA0910D03A53018F0E9
:101AE200E0E0E0930D030E94B32E20810E94AD2E10
:101AF200A0912303EFEF0E943536E02121F0E0911F
:101B02002303EF5F03C0E894F1F8E0E0E0932303DE
:101B1200A0912303A43109F06AC1AE81E0E00E94E2
:101B22002B360E2E0E943D2DE02119F0EE81E15060
:101B3200EE83233610F423E65AC121E0E0E0E0937D
:101B42000D03E0911503A0E0B0E00E947C2EE0912D
:101B52001603A1E0B0E00E947C2EE0911703A2E000
:101B6200B0E00E947C2EE0911903A3E0B0E00E9455
:101B72007C2EE8A5A4E0B0E00E947C2EE9A5A5E0B9
:101B8200B0E00E947C2EEAA5A6E0B0E00E947C2E86
:101B9200E0911A03A7E0B0E00E947C2EE0911B03C3
:101BA200A8E0B0E00E947C2EE0911F03A9E0B0E023
:101BB2000E947C2EE0912403AAE0B0E00E947C2ED9
:101BC2000E94212CA2E3B0E00E94602EECA1A3E1CE
:101BD200B0E00E947C2EEDA1A4E1B0E00E947C2E38
:101BE200EEA1A5E1B0E00E947C2EE8A1ABE0B0E05E
:101BF2000E947C2EE9A1ACE0B0E00E947C2EEAA11A
:101C0200ADE0B0E00E947C2EE989FA89A6E3B0E05B
:101C12000E94602EE0913103AEE0B0E00E947C2E83
:101C2200E0913303AFE0B0E00E947C2EE0913203FA
:101C3200A0E1B0E00E947C2EE32FA1E1B0E00E947F
:101C42007C2EED89FE89A8E3B0E00E94602EEBA510
:101C5200A2E1B0E00E947C2EEB85FC85A8E4B0E016
:101C62000E94602E0E94662E0E94B92EACE3B0E064
:101C72000E94602EE0916E03F0916F03A0E4B0E049
:101C82000E94602EE0E023FCE1E0A6E1B0E00E94C9
:101C92007C2E0E94702BAEE3B0E00E94602EE09199
:101CA2000603A7E1B0E00E947C2EE0910803A8E1C0
:101CB200B0E00E947C2EE0910903A9E1B0E00E940D
:101CC2007C2EE0910A03AAE1B0E00E947C2EE09112
:101CD2000B03ABE1B0E00E947C2EE0910C03ACE17F
:101CE200B0E00E947C2E0E949B2A0E944D2B0E94F3
:101CF200732EE0912803ADE1B0E00E947C2EE091CA
:101D02002903AEE1B0E00E947C2EE0912A03AFE10C
:101D1200B0E00E947C2EE0912B03A0E2B0E00E9492
:101D22007C2EE0912C03A1E2B0E00E947C2EE09197
:101D32002D03A2E2B0E00E947C2EE0912E03A3E2EA
:101D4200B0E00E947C2EE0912F03A4E2B0E00E945A
:101D52007C2E0E94782EE0910E03A5E2B0E00E9454
:101D62007C2EE0E036FCE1E0A6E2B0E00E947C2EB0
:101D7200E0911003A9E2B0E00E947C2EEB8DAAE272
:101D8200B0E00E947C2EED85FE85A6E4B0E00E94C4
:101D9200602EE0913C03ABE2B0E00E947C2EE09129
:101DA2003D03ACE2B0E00E947C2EE0913E03ADE246
:101DB200B0E00E947C2EE0911C03AEE2B0E00E94F3
:101DC2007C2EE0911E03AFE2B0E00E947C2EE091F7
:101DD2002003A0E3B0E00E947C2EE0912103A1E366
:101DE200B0E00E947C2E0E94392BE1E04E2E0E9430
:101DF200AD2EA0E0F1FCA1E00E94642DAE81E4E6EC
:101E02000E9426360E94512E51F06894F1F8EE811C
:101E1200EF5FEE83AE81A43611F4E0E0EE83EAE0F8
:101E2200E61510F4E894F0F80E94372DA0E0F0FCDB
:101E3200A1E00E94642DAE81E0E00E9421360E9462
:101E4200512E51F06894F0F8EE81E150EE83AE81AC
:101E5200AF3F11F4E3E6EE830E94852C0E94BE2E72
:101E6200C1F00E94C42EA9F4A0913803A43119F440
:101E7200E7E0E0933803E0E0E0933903E894F3F815
:101E8200A0913803A33028F0E0913803E150E093A9
:101E92003803AB2DEAE00E9435360E2E0E94BE2E8C
:101EA200C1F00E94C42EA9F4A0913803A43119F400
:101EB200E7E0E0933803E0E0E0933903E894F2F8D6
:101EC200A0913803A33028F0E0913803E150E09369
:101ED2003803AB2D0E94822EAA2DEAE00E943A36E8
:101EE200E02131F0E0E0E0933903E4E1E0933803EC
:101EF200EAE0EA1510F4E894F3F80E94852C0E94B7
:101F02008B2C0E941736E02109F4F2C26894F3F890
:101F1200AE81A13049F4A0911503A13028F4E091DB
:101F22001503EF5FE0931503AE81A23049F4A0914F
:101F32001603A23328F4E0911603EB5FE093160335
:101F4200AE81A33049F4A0911703A43628F4E0919E
:101F52001703EF5FE0931703AE81A43049F4A09119
:101F62001903A83228F4E0911903EF5FE0931903F3
:101F7200AE81A53031F4A8A5A43618F4E8A5EF5F28
:101F8200E8A7AE81A63031F4A9A5A43618F4E9A5D4
:101F9200EF5FE9A7AE81A73031F4AAA5A43618F401
:101FA200EAA5EF5FEAA7AE81A83049F4A0911A032F
:101FB200AF3F28F4E0911A03EF5FE0931A03AE817A
:101FC200A93049F4A0913C03AF3F28F4E0913C03CF
:101FD200EF5FE0933C03AE81AA3049F4A0913D0348
:101FE200AF3F28F4E0913D03EF5FE0933D03AE8104
:101FF200AB3049F4A0913E03AF3F28F4E0913E0399
:10200200EF5FE0933E03AE81AC3049F4A0910E0342
:10201200A03328F4E0910E03E45FE0930E03AE8157
:10202200AD3069F4A0914E03B0914F03A83BEBE0B1
:10203200BE0728F40E94212C31960E94BA2BAE8151
:10204200AE3031F4ACA1A43618F4ECA1EB5FECA3F2
:10205200AE81AF3031F4ADA1A43618F4EDA1EB5F3F
:10206200EDA3AE81A03131F4AEA1A43618F4EEA1F5
:10207200EB5FEEA3AE81A13131F4A8A1A83C18F424
:10208200E8A1EB5FE8A3AE81A23131F4A9A1A83C9B
:1020920018F4E9A1EB5FE9A3AE81A33131F4AAA15F
:1020A200A83C18F4EAA1EB5FEAA3AE81A43169F47B
:1020B200A0915E03B0915F03A835E2E0BE0728F469
:1020C2000E94702B7E960E94D42BAE81A53189F49A
:1020D200A0910E03EAE0EA9FF001EA5BFF4FA989B3
:1020E200BA89AE17BF0728F4E989FA893196E98BD4
:1020F200FA8BAE81A63149F4A0913103A13028F4C4
:10210200E0913103EF5FE0933103AE81A73149F4EF
:10211200A0913303A23328F4E0913303EF5FE093FD
:102122003303AE81A83149F4A0913203A13028F4DF
:10213200E0913203EF5FE0933203AE81A93181F483
:10214200A32FE4E10E94CF2E0E94692D09F03F5F88
:10215200A32FEEE10E94CF2E0E94452E09F03F5F91
:10216200AE81AA3159F40E94D62EAC3BE2E0BE0702
:1021720028F40E94B92E31960E94C62BAE81AB3153
:1021820091F40E94AD2AA73EE3E0BE07E0E08E078D
:10219200E0E09E0740F40E94702AEF5FFF4F6F4F0E
:1021A2007F4F0E94CB2BAE81AC3161F4A0E023FCC7
:1021B200A1E0A13038F4E0E023FCE1E0EF5F0E940F
:1021C200BD3723F8AE81AD3169F40E94302AAE3DAD
:1021D200E3E0BE0738F40E94112A3A96E0935603D0
:1021E200F0935703AE81AE3169F40E943A2AA835C2
:1021F200E2E0BE0738F40E941D2A3A96E093620399
:10220200F0936303AE81AF3149F4A0910603AA3083
:1022120028F4E0910603EF5FE0930603AE81A0325B
:1022220049F4A0910803AB3028F4E0910803EF5F72
:10223200E0930803AE81A13249F4A0910903AB30C7
:1022420028F4E0910903EF5FE0930903AE81A23223
:1022520049F4A0910A03AB3028F4E0910A03EF5F3E
:10226200E0930A03AE81A33249F4A0910B03AB3091
:1022720028F4E0910B03EF5FE0930B03AE81A432ED
:1022820049F4A0910C03AB3028F4E0910C03EF5F0A
:10229200E0930C03AE81A53249F4A0912803A1304A
:1022A20028F4E0912803EF5FE0932803AE81A63281
:1022B20049F4A0912903A13028F4E0912903EF5FAA
:1022C200E0932903AE81A73249F4A0912A03A230F8
:1022D20028F4E0912A03EF5FE0932A03AE81A8324B
:1022E20049F4A0912B03A13028F4E0912B03EF5F76
:1022F200E0932B03AE81A93249F4A0912C03A230C2
:1023020028F4E0912C03EF5FE0932C03AE81AA3214
:1023120049F4A0912D03A33028F4E0912D03EF5F3F
:10232200E0932D03AE81AB3249F4A0912E03A1308C
:1023320028F4E0912E03EF5FE0932E03AE81AC32DE
:1023420049F4A0912F03A13028F4E0912F03EF5F0D
:10235200E0932F03AE81AD3291F40E943F2BAF394F
:10236200E6E8BE07E1E08E07E0E09E0740F40E9447
:10237200272BE65FFF4F6F4F7F4F0E94302BAE81BE
:10238200AE3259F40E94DB2EA031E7E2BE0728F4F8
:102392000E94912A3A960E94962AAE81AF3261F447
:1023A200A0E036FCA1E0A13038F4E0E036FCE1E048
:1023B200EF5F0E94BD3736F8AE81A03349F4A09199
:1023C2001003A13028F4E0911003EF5FE0931003B3
:1023D200AE81A13331F4AB8DA33018F4EB8DEF5FF6
:1023E200EB8FAE81A23359F4AD85BE85A632E2E011
:1023F200BE0728F4ED85FE853196ED87FE87AE8116
:10240200AC3549F4A0910503AA3F28F4E0910503F5
:10241200EB5FE0930503AE81AD3531F4ACA5A93095
:1024220018F4ECA5EF5FECA7AE81AE3559F4AD8997
:10243200BE89A83BEBE0BE0728F4ED89FE89319600
:10244200ED8BFE8BAE81AF3531F4ABA5AA3018F41B
:10245200EBA5EF5FEBA7AE81A03659F4AB85BC8547
:10246200A83EE3E0BE0728F4EB85FC853A96EB87AD
:10247200FC87AE81A13649F4A0912403AC3328F441
:10248200E0912403EF5FE0932403AE81A23691F43E
:102492000E94972EA081AA3F21F40E94E02EEB5FBA
:1024A200EC930E94972EA081AA3F20F40E94E02E76
:1024B200E65FEC930E94E72E0E945736E02149F036
:1024C200A0911B03AA3F28F4E0911B03E65FE0936F
:1024D2001B030E94E72E0E946336E02149F0A0917F
:1024E2001C03AA3F28F4E0911C03E65FE0931C035F
:1024F200EAE0EB1510F4E894F2F8AB2DEAE00E9462
:1025020035360E2EA0E0F2FCA1E00E94642D0E945E
:10251200BE2E09F4E2C26894F2F8AE81A13049F409
:10252200A0911503A13028F0E0911503E150E0934A
:102532001503AE81A23049F4A0911603AB3028F006
:10254200E0911603E550E0931603AE81A33049F4FF
:10255200A0911703AD3328F0E0911703E150E09307
:102562001703AE81A43049F4A0911903A53128F0D4
:10257200E0911903E150E0931903AE81A53031F4E3
:10258200A8A5A13018F0E8A5E150E8A7AE81A630D1
:1025920031F4A9A5A13018F0E9A5E150E9A7AE816F
:1025A200A73031F4AAA5A13018F0EAA5E150EAA7B4
:1025B200AE81A83049F4A0911A03A13028F0E0912D
:1025C2001A03E150E0931A03AE81A93049F4A091B5
:1025D2003C03A13028F0E0913C03E150E0933C033E
:1025E200AE81AA3049F4A0913D03A13028F0E091D8
:1025F2003D03E150E0933D03AE81AB3049F4A0913D
:102602003E03A13028F0E0913E03E150E0933E0307
:10261200AE81AC3049F4A0910E03A93128F0E091CB
:102622000E03EC50E0930E03AE81AD3069F4A0913D
:102632004E03B0914F03A93EE3E0BE0728F00E948B
:10264200212C31970E94BA2BAE81AE3031F4ACA16D
:10265200A63018F0ECA1E550ECA3AE81AF3031F416
:10266200ADA1A63018F0EDA1E550EDA3AE81A031E9
:1026720031F4AEA1A63018F0EEA1E550EEA3AE8182
:10268200A13131F4A8A1A13018F0E8A1E550E8A3E6
:10269200AE81A23131F4A9A1A13018F0E9A1E5502F
:1026A200E9A3AE81A33131F4AAA1A13018F0EAA1C5
:1026B200E550EAA3AE81A43161F4A0915E03B0912A
:1026C2005F030E94A93728F40E94702B7E970E9414
:1026D200D42BAE81A53189F4A0910E03EAE0EA9FE2
:1026E200F001E654F040A989BA89EA17FB0728F4F9
:1026F200E989FA893197E98BFA8BAE81A63149F4DF
:10270200A0913103A13028F0E0913103E150E09330
:102712003103AE81A73149F4A0913303A23028F0EE
:10272200E0913303E150E0933303AE81A83149F4E1
:10273200A0913203A13028F0E0913203E150E093FE
:102742003203AE81A93119F4323008F03150AE8132
:10275200AA3159F40E94D62EA935E2E0BE0728F02C
:102762000E94B92E31970E94C62BAE81AB3191F4F3
:102772000E94AD2AAB30E0E0BE07E0E08E07E0E069
:102782009E0740F00E94702AE150F0406040704085
:102792000E94CB2BAE81AC3159F4A0E023FCA1E026
:1027A200A13030F0A0E023FCA1E00E94ED2E23F83E
:1027B200AE81AD3161F40E94302A0E94A93738F40B
:1027C2000E94112A3197E0935603F0935703AE818A
:1027D200AE3161F40E943A2A0E94A93738F40E946D
:1027E2001D2A3197E0936203F0936303AE81AF3108
:1027F20049F4A0910603A23028F0E0910603E150CB
:10280200E0930603AE81A03249F4A0910803A230FE
:1028120028F0E0910803E150E0930803AE81A13271
:1028220049F4A0910903A13028F0E0910903E15095
:10283200E0930903AE81A23249F4A0910A03A130C8
:1028420028F0E0910A03E150E0930A03AE81A3323B
:1028520049F4A0910B03A13028F0E0910B03E15061
:10286200E0930B03AE81A43249F4A0910C03A13092
:1028720028F0E0910C03E150E0930C03AE81A53205
:1028820049F4A0912803A13028F0E0912803E150F7
:10289200E0932803AE81A63249F4A0912903A13026
:1028A20028F0E0912903E150E0932903AE81A73299
:1028B20049F4A0912A03A13028F0E0912A03E150C3
:1028C200E0932A03AE81A83249F4A0912B03A130F0
:1028D20028F0E0912B03E150E0932B03AE81A93263
:1028E20049F4A0912C03A13028F0E0912C03E1508F
:1028F200E0932C03AE81AA3249F4A0912D03A130BA
:1029020028F0E0912D03E150E0932D03AE81AB322C
:1029120049F4A0912E03A13028F0E0912E03E1505A
:10292200E0932E03AE81AC3249F4A0912F03A13083
:1029320028F0E0912F03E150E0932F03AE81AD32F6
:1029420069F40E943F2B0E94AD3740F40E94272B6E
:10295200E150F040604070400E94302BAE81AE32B8
:1029620051F40E94DB2E0E94A93728F40E94912A7A
:1029720031970E94962AAE81AF3259F4A0E036FC1C
:10298200A1E0A13030F0A0E036FCA1E00E94ED2EE3
:1029920036F8AE81A03349F4A0911003A13028F09B
:1029A200E0911003E150E0931003AE81A13331F4C2
:1029B200AB8DA13018F0EB8DE150EB8FAE81A233DD
:1029C20059F4AD85BE85A93CE0E0BE0728F0ED854F
:1029D200FE853197ED87FE87AE81AC3549F4A09133
:1029E2000503A13028F0E0910503E550E0930503CB
:1029F200AE81AD3531F4ACA5A13018F0ECA5E150B3
:102A0200ECA7AE81AE3559F4AD89BE89A13DE7E0B0
:102A1200BE0728F0ED89FE893197ED8BFE8BAE81E2
:102A2200AF3531F4ABA5A13018F0EBA5E150EBA71F
:102A3200AE81A03659F4AB85BC85A536E0E0BE0771
:102A420028F0EB85FC853A97EB87FC87AE81A136AF
:102A520049F4A0912403A13028F0E0912403E1502D
:102A6200E0932403AE81A236D1F40E94972EBF01D7
:102A7200A0810E94512BFB01A081EFEF0E9435360D
:102A8200E02121F00E94E02EEA50EC930E94972E62
:102A9200A081AF3F21F40E94E02EE550EC930E940A
:102AA200E72E0E945736E02149F0A0911B03A13086
:102AB20028F0E0911B03EA50E0931B030E94E72EEB
:102AC2000E946336E02149F0A0911C03A13028F056
:102AD200E0911C03EA50E0931C0323FC5CC0E091EC
:102AE2008803F0918903A0EEB3E00E94BF2B0E94FD
:102AF200F42EE0E0F0E06EEF72E40E94AB3509F0F4
:102B020008F40AC00E94FD2EA0E0B0E080E893E441
:102B12000E94C1340E94062FE0914303F0E0E0934B
:102B22008E03F0938F030E940F2FA038E0E0BE07C0
:102B320054F0E0918E03F0918F03E050F140E09366
:102B42008E03F0938F030E94F42E0E94AD373CF463
:102B52000E94142F0E94C8340E941A2F14C0A09100
:102B6200E303AA233AF40E94142F0E94C1340E9464
:102B72001A2F09C0E0E0E093D003E093D103E09381
:102B8200D203E093D3030E94232FA0E8B3E00E9474
:102B9200C52A0E94252F23FE47C0EF81F8850E9497
:102BA2000F2E0E9457370E945237E0E0F0E060E8B3
:102BB20074E40E946635A0E0B0E48CE995E40E94DA
:102BC2001835DF01CB01ED89FE89662777270E9440
:102BD2008E340E948C2ADF01CB01E3E3F3E365E844
:102BE20072E40E9466350E94062FA0910F03A13065
:102BF20048F4E0E0E093E003E093E103E093E203D2
:102C0200E093E3030E94FD2E0E941A2FE091060337
:102C1200A0910703AE1740F00E94232FA0E8B3E073
:102C22000E94C52A0E94252FA0E0F0FCA1E00E948C
:102C32006E2DE0910603A09107030E943036E02139
:102C420009F44DC0E0912B03E03021F5E0912A0315
:102C5200E03041F4A985BA85E0E0F4E00E94292F32
:102C62000E943B2FA0912A03A13041F4E0918A03F4
:102C7200F0918B030E943E2F0E943B2FA0912A03CA
:102C8200A23041F4E0918C03F0918D030E943E2F1B
:102C92000E943B2FA0912B03A130F1F4E0912A0373
:102CA200E03031F4AF81B8850E94452F0E944A2F4F
:102CB200A0912A03A13031F4E0918A03F0918B03B1
:102CC2000E944A2FA0912A03A23031F4E0918C0392
:102CD200F0918D030E944A2FE0E0E0930703F09108
:102CE2006403E0E0DF01E0913703F0E0EA0FFB1F4D
:102CF200A0EBB3E00E94162A0E944F2FA0E0B0E0A2
:102D020080E192E40E9466357F936F93FF93EF9385
:102D12000E94D62E0E94582FAF91BF918F919F9102
:102D2200662777270E948E340E941835E093B003FD
:102D3200F093B1036093B2037093B3030E945D2FCB
:102D4200E0E0F0E060E87FE30E94D1350E2E0E94C1
:102D52005D2FE0E0F0E068EC72E40E94CB35E02108
:102D620009F10E944F2FA0E0B0E080E09FE30E94B3
:102D7200C834A8E9B3E00E9457340E944D370E943C
:102D82004F2FE093B403F093B5036093B6037093AF
:102D9200B7030E945D2F0E944D2BA0E5B3E00E9475
:102DA200482A15C0E0E0E0939803E0939903E0938A
:102DB2009A03E0939B03E093B403E093B503E0939B
:102DC200B603E093B703E0935003E09351030E94EC
:102DD200D12A0E94482B0E94D135EF930E94662F80
:102DE2000E94D135AF91EA23C1F10E945E2AE0E050
:102DF200F0E068EC72E40E9466350E94AD2A0E94FF
:102E02005C370E948C2A0E94682FA091AC03B0917B
:102E1200AD038091AE039091AF03E0E0F0E064E196
:102E220072E40E941835DF01CB010E94E82A0E9459
:102E32006635A0E0B0E080E291E40E9418350E947D
:102E4200682FE091AC03F091AD036091AE037091F5
:102E5200AF03DE0114960E94C52A0E94372DA0916D
:102E62002203EDEF0E9435360E220E943D2DE02115
:102E720029F0E0912203EF5FE0932203A62D0E9446
:102E8200822EA0912203EFEF0E9435360E220E947D
:102E92003D2DE02129F0E894F0F8E0E0E0932203F0
:102EA200A0912203EEE10E9417360E2E0E943D2DC4
:102EB200E02119F0E1E0E0932503E0912403E03002
:102EC20019F4E0E0E09325030E94562B0E94482B60
:102ED2000E9481360E94582EA09125030E94712FD4
:102EE20019F0E1E0E0932503A0912503AC3309F446
:102EF2001FEFA0910503A13020F0E09105030E948D
:102F02006F2CA0912F030E94822DA12F0E94712F5E
:102F120049F1EA8DEF5FEA8FF0E03196BF01A12F10
:102F2200B0E00E94FF2BE617F70784F40E94762F89
:102F32000E9471360E2E0E94832FE4EAF1E060E0D7
:102F420070E00E946936E02909F010E0A12FB0E09C
:102F52000E94FF2BAA8DB0E0EA17FB0714F4E0E011
:102F6200EA8F02C0E0E0EA8FA12F0E94512B0E945B
:102F7200762F0E9481360E22AD85BE85E4EAF1E00D
:102F82000E944536E02119F0163908F416E9EB8D56
:102F9200E03009F074C04420A9F4E02FF0E0349648
:102FA2000E948C2FAEE30E94F229A4E00E94F22933
:102FB200A02F0E94982FA09144030E94F229A12FD2
:102FC2000E949D2FE1E0E41509F059C04424A0912C
:102FD2001703B0E00E94452FE0931803F0E0BC967F
:102FE200DF01E0911403F0E0AE0FBF1FE091150383
:102FF200F0E0AE0FBF1FE09116030E94A82FAE0FA4
:10300200BF1FE8A5F0E0AE0FBF1FE9A5F0E0AE0FCD
:10301200BF1FEAA5F0E0AE0FBF1FE0911A030E94A6
:10302200AF2FF0E0AE0FBF1FE0913E030E94BA2F18
:10303200AEE30E94F229ACE20E94C22FA0911603D5
:103042000E94F229A09118030E94CC2FA8A50E94E9
:10305200F229A9A50E94F229AAA50E94F229A0910B
:103062001A030E94F229A0913C030E94F229A09126
:103072003D030E94F229A0913E030E949D2FAB8D39
:10308200A33009F068C0442099F5E02FF0E03596AE
:10309200DF01E0913F03F0E0AE0FBF1FE09140037C
:1030A200F0E0AE0FBF1FE0914103F0E0EA0FFB1F1B
:1030B2000E948C2FAEE60E94F229A5E00E94F2291E
:1030C200A02F0E94F229A0913F030E94F229A09111
:1030D20040030E94F229A09141030E94F229A0918B
:1030E20044030E94F229A12F0E94982F0E94D22FFE
:1030F200E1E0E41581F54424E0911403F0E0BD968B
:10310200DF01E09115030E94AF2F0E94A82FAE0F9E
:10311200BF1FD296E0911A030E94BA2FAEE60E9418
:10312200F229ADE20E94C22FA0913D030E94F22932
:10313200A0913C030E94CC2FA2E30E94982FA0E012
:103142000E94F229A0911A030E94982FA0E00E94E7
:10315200982F0E94D22F233608F0F7C60E94B32E72
:103162002081A0913503A13048F420FC07C0A0E0E3
:10317200F799A1E0EA2FE295E07F19C0A0E0F79964
:10318200A1E0EA2FE295E07F0E2EA0E0F399A1E004
:10319200EA2FEE0FEE0F0E0EA0E0F499A1E0EA2F57
:1031A200EE0FA02DAE0FE0E0F599E1E0EA0FEDA7FA
:1031B200EAE00E94D92FEAE0DE01AD5BBF4FEC935B
:1031C2000E94DE2FDE01AB5BBF4FEC93EAE00E9470
:1031D200E42FEAE00E94E92FEAE00E94EE2F0E942B
:1031E200F32FE89435F8A0E031FCA1E00E94822D93
:1031F200A0E032FCA1E0E1E00E9417360E2AA0E036
:1032020034FCA1E0E1E00E941736E02911F020FA37
:1032120001C0E894F5F8E0912D03E03021F40E941A
:1032220015300E942630A0912D03A13081F4A0E038
:1032320022FCA1E0EA2FEE0FE75F0E2EA0E022FCB7
:10324200A1E0EA2FEE0FEE0FE00D0E943530A091C3
:103252002D03A23099F40E941530A0E022FCA1E0D7
:10326200EA2F0E9445300E0EA0E022FCA1E0EA2FD8
:10327200E295E07FEE0F0E0E0E942630A0912D0304
:10328200A33031F4E0E022FCE1E0E85F0E94353057
:10329200A0910E03A83109F041C00E944A30A23D1C
:1032A200E0E0BE07E0E08E07E0E09E071CF0E1E010
:1032B200E09301030E945830A83FE0E0BE07E0E03F
:1032C2008E07E0E09E071CF0E3E0E09301030E941A
:1032D2005830AF3FE0E0BE07E0E08E07E0E09E0737
:1032E2001CF0E7E0E09301030E945830A430E1E0D3
:1032F200BE07E0E08E07E0E09E071CF0EFE0E093FF
:1033020001030E945830AE30E1E0BE07E0E08E07D4
:10331200E0E09E071CF0EFE1E0930103A0910E03B1
:10332200A43209F041C00E944A30A633E1E0BE0750
:10333200E0E08E07E0E09E071CF0E1E0E09301038D
:103342000E945830AA34E1E0BE07E0E08E07E0E0D8
:103352009E071CF0E3E0E09301030E945830AE3573
:10336200E1E0BE07E0E08E07E0E09E071CF0E7E048
:10337200E09301030E945830A836E1E0BE07E0E086
:103382008E07E0E09E071CF0EFE0E09301030E944D
:103392005830AC37E1E0BE07E0E08E07E0E09E0780
:1033A2001CF0EFE1E0930103A0910E03A03309F0BA
:1033B20041C00E944A30A638E1E0BE07E0E08E0735
:1033C200E0E09E071CF0E1E0E09301030E94583028
:1033D200AC3CE1E0BE07E0E08E07E0E09E071CF0B7
:1033E200E3E0E09301030E945830A63DE1E0BE070E
:1033F200E0E08E07E0E09E071CF0E7E0E0930103C7
:103402000E945830A03EE1E0BE07E0E08E07E0E017
:103412009E071CF0EFE0E09301030E945830AF3E9C
:10342200E1E0BE07E0E08E07E0E09E071CF0EFE17E
:10343200E0930103A0910203A431F0F40E94562B01
:103442000E9461306CF0FE01EF5BFF4F3396FF93F9
:10345200EF930E9469300E946F30AF91BF91EC935D
:103462000E947A30FF93EF930E9469300E941837CE
:10347200AF91BF91EC930DC020FE05C0E0E40E9425
:103482007F30E0E402C00E94DE2FDE01AB5BBF4F63
:10349200EC93A98DA13050F0E98DE150E98FE8E776
:1034A2000E947F30FE01EF5BFF4F0483A88DA130A5
:1034B20058F0E88DE150E88FE8E30E947F300E94E7
:1034C2007A30A0913003A083AF89A13058F0EF8900
:1034D200E150EF8BE9E30E947F30E0E5DE01AB5B78
:1034E200BF4FEC93E0911103E03029F5EEA5E058CF
:1034F200EEA7A0918103AA2392F4E0E40E94D92FBF
:10350200A0918003B0918103AD39EFEFBE0714F4AF
:10351200689435F80E9484300E948C3002C0E8948E
:1035220035F80E9491301A9724F00E9496300E943A
:103532009D300E94A530A0911103A13009F048C02E
:10354200EDA5E85FEDA7A0918703AA23A2F4E0E42A
:103552000E94D92F0E94B230A73FEFEFBE0714F4AA
:10356200689401C0E89435F8E0918603F0918703EE
:103572000E94E13506C0E89435F8E0918603F091A7
:103582008703E0938203F09383030E9491301A979A
:1035920024F00E9496300E949D300E94A5300E9425
:1035A200B230E3E6F0E00E9451360E2E0E94B230B5
:1035B200EDE9FFEF0E944B36E02951F0E89435F82F
:1035C200E0E40E94D92FE0E4DE01AD5BBF4FEC9353
:1035D2000E94B730FF93EF930E9458300E94BC3094
:1035E2000E946F30AF91BF910E94C1303696FF9317
:1035F200EF930E94C6300E946F30AF91BF910E943C
:10360200C1303796FF93EF930E94C6300E9418375D
:10361200AF91BF91EC930E945830A639E0E0BE070B
:10362200E0E08E07E0E09E0764F4E0E40E94E42F0D
:10363200E0E40E94E92FE0E40E94EE2FE0E0E09354
:103642000103213009F062C00E94CC300E94D630C2
:10365200A83EE3E0BE07C8F0EFA5E05EEFA70E9438
:10366200DB300E94E1300E94C1303E96BF010E94D1
:10367200D6300E94EC300E94C1303F96BF010E94BA
:10368200D6300E94582FDF011DC0EFA5E056EFA7EC
:103692000E94D630A436E0E0BE0728F00E94DB305C
:1036A2000E94EC30EC930E94F730BF010E94D630AA
:1036B2000E94582F0E94FC300E94C1303F96BF01E9
:1036C2000E94D630EAE0F0E00E940331A0910003AC
:1036D200AA3010F00E940831FE01EF5BFF4F3996CD
:1036E200BF01A09100030E940E310E94C1303A96A0
:1036F200BF01AC2DB0E00E94FF2B0E949D300E94C2
:103702001531BF01AC2D0E940E31EC93223009F02D
:103712006FC0EFA5E05CEFA70E943F2BA03AE6E85E
:10372200BE07E1E08E07E0E09E0778F00E941A31C2
:10373200FF93EF930E943F2BE0EAF6E861E070E02E
:103742000E941F31AF91BF91EC930E943F2B0E94C8
:103752002A3178F00E941531FF93EF930E943F2B9C
:10376200E0E1F7E260E070E00E941F31AF91BF91AB
:10377200EC930E943F2B0E94323168F00E943A3152
:10378200FF93EF930E943F2B0E942B2D0E941F312B
:10379200AF91BF91EC930E943F2B0E943F3168F0A2
:1037A2000E944731FF93EF930E943F2B0E94BC304F
:1037B2000E941F31AF91BF91EC930E943F2B0E9458
:1037C200613058F00E94F730FF93EF930E944C3122
:1037D2000E941F31AF91BF91EC930E945231FF932F
:1037E200EF930E944C310E941437AF91BF91EC933A
:1037F200233009F08FC0E7E70E945731A091A70359
:10380200AA2392F4E091A403F091A5036091A60388
:103812007091A7030E94E535E093A403F093A503FA
:103822006093A6037093A7030E94662F0E948C2ABE
:10383200772312F40E9461310E94662F0E948C2A23
:103842000E94673110F40E9470310E94662F0E941C
:103852008C2A0E94763110F40E947F310E94662FDA
:103862000E948C2A0E94853110F40E9488310E94A5
:103872008E310E942A317CF00E941531FF93EF9322
:103882000E948E31E0E1F7E260E070E00E946F306A
:10389200AF91BF91EC930E948E310E9432316CF055
:1038A2000E943A31FF93EF930E948E310E942B2D9A
:1038B2000E946F30AF91BF91EC930E948E310E94B3
:1038C2003F316CF00E944731FF93EF930E948E319B
:1038D2000E94BC300E946F30AF91BF91EC930E9466
:1038E2008E310E9461305CF00E94F730FF93EF93BB
:1038F2000E9497310E946F30AF91BF91EC930E946A
:103902005231FF93EF930E9497310E941837AF9183
:10391200BF91EC93243009F052C00E949D31A091D6
:103922007D03AA2312F40E94A2310E94AD317723B3
:1039320012F40E9461310E94AD310E94673110F48D
:103942000E9470310E94AD310E94763110F40E94C3
:103952007F310E94AD310E94853110F40E9488317E
:103962000E94B331A031E7E2BE0724F00E94153174
:103972000E94B8310E94B331A83EE3E0BE0724F0B2
:103982000E943A310E94BF310E94B331A436E0E076
:10399200BE0724F00E9447310E94C6310E94B33113
:1039A2001A974CF00E94F730BF010E94B3310E9477
:1039B200FF2B0E949D300E9452310E94CD31253052
:1039C20061F50E949D310E94D631A091D703AA23AE
:1039D20012F40E9470310E94D12AE0E0F0E066EC1D
:1039E20072EC0E94AB3510F40E947F310E94DC31F0
:1039F200A436E0E0BE0724F00E9447310E94E13184
:103A02000E94F730BF010E94DC310E94FF2B0E940E
:103A12009D300E9452310E94E8312630E1F5EFA537
:103A2200E058EFA7E0E00E94F131E5E00E94F631B4
:103A3200E8E70E94FB31AC81BD81A83EE3E0BE070E
:103A42004CF00E943A31BF01AC81BD81E8EEF3E057
:103A52000E940032AC81BD81A436E0E0BE074CF08A
:103A62000E944731BF01AC81BD81E4E6F0E00E94D3
:103A720000320E94F730BF01AC81BD810E94FF2B52
:103A82000E949D300E945231BF01AC81BD810E94D3
:103A92000332DB01EC93273009F057C0113040F1BB
:103AA200ECE00E94F1310E940832E436A0E0FA070D
:103AB2004CF00E941A31BF01A12FB0E0E8ECF0E017
:103AC2000E9400320E9408323A974CF00E9415314F
:103AD200BF01A12FB0E0E4E1F0E00E9400320E94B9
:103AE2003A31BF010E940832DF010E9403322BC02B
:103AF200EBE00E94F1310E940B32E436A0E0FA07BB
:103B020050F00E941A31BF01AF85B889E8ECF0E0AD
:103B12000E941032EC930E940B323A9750F00E94AE
:103B22001531BF01AF85B889E4E1F0E00E9410329F
:103B3200EC930E943A31BF010E940B32DF01EAE0AE
:103B4200F0E00E940337DB01EC93283009F081C0DA
:103B52000E94CC30A0917803B0917903A135EBEFAC
:103B6200BE0734F4E1E5FBEFE0937803F0937903C9
:103B7200A0917803B0917903A03BE4E0BE0734F052
:103B8200EFEAF4E0E0937803F0937903A0917903EC
:103B9200AA234AF40E947F31E0917803F0917903DD
:103BA2000E94E13504C0E0917803F0917903E0933B
:103BB2007A03F0937B03A0917A03B0917B03ECE349
:103BC200F0E00E94D436E0935803F09359030E9428
:103BD2001332ECE30E94B136A0917A03B0917B03D9
:103BE200AE1BBF0BA0935A03B0935B0324FE28C005
:103BF2000E9413321A9710F00E940831FE01EF5B07
:103C0200FF4F3996BF010E941332EAE0F0E00E94B2
:103C12000337DB010E94C1303A96BF01A0915A03DB
:103C2200B0915B030E94582F0E94FC300E94C13069
:103C32003B96BF01A0915A03B0915B030E941832D8
:103C4200E3E70E941B32E8E30E942032E4E50E948F
:103C52002532293009F058C0EFA5E058EFA70E949D
:103C62000831EEE30E945731A0917D03AA2312F49A
:103C72000E94A2310E94AD31772312F40E94613179
:103C82000E94AD310E94673110F40E9470310E948F
:103C9200AD310E94763110F40E947F310E94AD3125
:103CA2000E94853110F40E9488310E94B331A03104
:103CB200E7E2BE0724F00E9415310E94B8310E944B
:103CC200B331A83EE3E0BE0724F00E943A310E94DD
:103CD200BF310E94B331A436E0E0BE0724F00E9457
:103CE20047310E94C6310E94B3311A974CF00E94AC
:103CF200F730BF010E94B3310E94FF2B0E949D301A
:103D02000E9452310E94CD312A3009F5EFA5E058C8
:103D1200EFA70E940831EEE30E9457310E94D6318C
:103D22000E94DC31A436E0E0BE0724F00E94473155
:103D32000E94E1310E94F730BF010E94DC310E94F3
:103D4200FF2B0E949D300E9452310E94E8312B309D
:103D5200B1F5EFA5E054EFA7E9E30E94F631E8E3FD
:103D62000E94FB310E94DB2EA83EE3E0BE0740F03A
:103D72000E943A31BF010E94DB2E0E94E130EC9397
:103D82000E94DB2EA436E0E0BE0740F00E944731DD
:103D9200BF010E94DB2E0E94EC30EC930E94F730B0
:103DA200BF010E94DB2E0E94582F0E94FC300E940D
:103DB200C1303F96BF010E94DB2E0E941832AE8DA9
:103DC2000E94512BAD8DE0E00E943A36E02909F4C1
:103DD200B5C0EFA5EF77EFA7E0913603E170EE0FE4
:103DE200AEA5EA23EEA7E0913603E6950E942A32B9
:103DF2000E2EE0913603E695E695E170AE2FE0E0F7
:103E0200F5FCE1E0EA2BEE0FEE0FE00DAEA5EA0FB6
:103E1200EEA70E94F32FAD8D0E94512BAE8D0E9412
:103E2200712F59F1AD8DA13029F40E942F32ECE0AF
:103E32000E943232AD8DA23029F40E942F32EDE081
:103E42000E943232AD8DA33029F40E942F32EBE072
:103E52000E9432320E94373229F00E942F32ECE067
:103E62000E9432320E94802C0E94413229F00E942C
:103E72002F32EBE00E9432322AC0AD8DA13029F4FC
:103E82000E944732ECE00E942532AD8DA23029F427
:103E92000E944732EDE00E942532AD8DA33029F415
:103EA2000E944732EBE00E9425320E94373229F00D
:103EB2000E944732ECE00E9425320E94802C0E9430
:103EC200413229F00E944732EBE00E942532AE8D4A
:103ED200A13029F40E944B32ECE00E942532AE8DD3
:103EE200A23029F40E944B32EDE00E942532AE8DC1
:103EF200A33029F40E944B32EBE00E942532AE8DB2
:103F0200E4E00E9417360E94413229F00E944B32AF
:103F1200ECE00E942532AE8DE5E00E9417360E9449
:103F2200413229F00E944B32EBE00E942532E091AF
:103F32001103E03019F4EEA5E058EEA7F29B05C09C
:103F4200EEA5EB7FEEA7EF5FEEA7233609F0A4C63E
:103F520051E0503140F40E944F32EAE0EC93E89491
:103F620035F85F5FF6CFAE81EBE50E945732EAE5A6
:103F72000E941736E02911F0E2E3EE83AE81A3330B
:103F820011F4ECE5EE83EE81E03029F4E0911403C4
:103F9200F0E0EB8BFC8BAE81A13029F4E0911503AC
:103FA200F0E0EB8BFC8BAE81A23029F4E09116039A
:103FB200F0E0EB8BFC8BAE81A33029F4E091170388
:103FC200F0E0EB8BFC8BAE81A43029F4E091190375
:103FD200F0E0EB8BFC8BAE81A53021F4E8A5F0E09C
:103FE200EB8BFC8BAE81A63021F4E9A5F0E0EB8BE4
:103FF200FC8BAE81A73021F4EAA5F0E0EB8BFC8BC1
:10400200AE81A83029F4E0911A03F0E0EB8BFC8B2F
:10401200AE81A93029F4E0913C03F0E0EB8BFC8BFC
:10402200AE81AA3029F4E0913D03F0E0EB8BFC8BEA
:10403200AE81AB3029F4E0913E03F0E0EB8BFC8BD8
:10404200AE81AC3029F4E0910E03F0E0EB8BFC8BF7
:10405200AE81AD3021F40E94212CEB8BFC8BAE8122
:10406200AE3021F4ECA1F0E0EB8BFC8BAE81AF30F3
:1040720021F4EDA1F0E0EB8BFC8BAE81A03121F4B9
:10408200EEA1F0E0EB8BFC8BAE81A13121F4E8A133
:10409200F0E0EB8BFC8BAE81A23121F4E9A1F0E0E0
:1040A200EB8BFC8BAE81A33121F4EAA1F0E0EB8B28
:1040B200FC8BAE81A43121F40E94702BEB8BFC8B24
:1040C200AE81A53121F4E989FA89EB8BFC8BAE81B3
:1040D200A63129F4E0913103F0E0EB8BFC8BAE8149
:1040E200A73129F4E0913303F0E0EB8BFC8BAE8136
:1040F200A83129F4E0913203F0E0EB8BFC8BAE8126
:10410200A93121F4E32FF0E0EB8BFC8BAE81AA31D5
:1041120021F40E94B92EEB8BFC8BAE81AB3131F4D2
:10412200E0916E03F0916F03EB8BFC8BAE81AC31AF
:1041320031F4E0E023FCE1E0F0E0EB8BFC8BAE81BC
:10414200AD3121F40E94112AEB8BFC8BAE81AE3192
:1041520021F40E941D2AEB8BFC8BAE81AF3129F436
:10416200E0910603F0E0EB8BFC8BAE81A03229F4E8
:10417200E0910803F0E0EB8BFC8BAE81A13229F4D5
:10418200E0910903F0E0EB8BFC8BAE81A23229F4C3
:10419200E0910A03F0E0EB8BFC8BAE81A33229F4B1
:1041A200E0910B03F0E0EB8BFC8BAE81A43229F49F
:1041B200E0910C03F0E0EB8BFC8BAE81A53229F48D
:1041C200E0912803F0E0EB8BFC8BAE81A63229F460
:1041D200E0912903F0E0EB8BFC8BAE81A73229F44E
:1041E200E0912A03F0E0EB8BFC8BAE81A83229F43C
:1041F200E0912B03F0E0EB8BFC8BAE81A93229F42A
:10420200E0912C03F0E0EB8BFC8BAE81AA3229F417
:10421200E0912D03F0E0EB8BFC8BAE81AB3229F405
:10422200E0912E03F0E0EB8BFC8BAE81AC3229F4F3
:10423200E0912F03F0E0EB8BFC8BAE81AD3231F4D9
:10424200E0916A03F0916B03EB8BFC8BAE81AE3293
:1042520021F40E94912AEB8BFC8BAE81AF3231F4B8
:10426200E0E036FCE1E0F0E0EB8BFC8BAE81A033CA
:1042720029F4E0911003F0E0EB8BFC8BAE81A133CB
:1042820021F4EB8DF0E0EB8BFC8BAE81A23321F4B9
:10429200ED85FE85EB8BFC8BAE81AC3529F4E0918C
:1042A2000503F0E0EB8BFC8BAE81AD3521F4ECA580
:1042B200F0E0EB8BFC8BAE81AE3521F4ED89FE890B
:1042C200EB8BFC8BAE81AF3521F4EBA5F0E0EB8BF1
:1042D200FC8BAE81A03621F4EB85FC85EB8BFC8B4D
:1042E200AE81A13629F4E0912403F0E0EB8BFC8B44
:1042F200AE81A23631F40E94972EE081F0E0EB8B82
:10430200FC8B0E94E72E0E945736E02129F0E091B3
:104312001B03F0E0EB8BFC8B0E94E72E0E946336BE
:10432200E02129F0E0911C03F0E0EB8BFC8BAE81E5
:104332000E946E2DAE81E3E00E945C32E1E10E94B8
:104342005C32E2E10E945C32E3E10E945C32E5E130
:104352000E945C32EBE10E945C32EDE10E945C3231
:10436200EEE20E941736E0291E2E0E9461320E9460
:104372004536E021E12911F0F69A01C0F698A0E055
:10438200F699A1E0EA2FE795E0E0E795EFA7E0E0F4
:10439200EEA7EDA7E0930103FE01EF5BFF4F33961B
:1043A200BF01AE81B0E0A7FDBFEF0E94FF2B0E94CC
:1043B2009D300E947A30BF01AE81B0E0A7FDBFEF11
:1043C2000E940332DB01EC93AB89BC89A031E7E2A6
:1043D200BE0750F00E941531BF01AB89BC89E0E1F4
:1043E200F7E20E941032EC93AB89BC89A83EE3E06D
:1043F200BE0740F00E943A31BF01AB89BC890E94DE
:10440200E130EC93AB89BC89A436E0E0BE0740F012
:104412000E944731BF01AB89BC890E94EC30EC930A
:10442200AB89BC891A9738F00E94F7300E946B3230
:104432000E94FC30EC930E945231BF01AB89BC89CF
:104442000E941832EE81E03079F4ECE10E946F3282
:10445200E0E50E94EE2FEDE60E94F631E4E50E94CF
:10446200FB31E0E50E943232AE81A13031F4EBE55E
:104472000E946F32EDE60E94EE2FAE81A23049F427
:10448200EDE60E94E42FE3E70E94E92FE8E30E94B1
:10449200EE2FAE81A33049F4EEE50E94E42FE0E373
:1044A2000E94E92FE7E70E94EE2FAE81A83011F4B7
:1044B2000E947232AE81AC3031F4EEE30E94783267
:1044C200ECE70E94EE2FAE81E1E10E945732E2E179
:1044D2000E945C32E3E10E945C32E5E10E945C32C0
:1044E200EDE10E945C32EEE20E941736E02939F0DB
:1044F2000E94F7300E946B320E94FC30EC93E7EA94
:10450200E0937A000E943D2CE7E2E0937A000E9459
:104512007B32EEE00E945C32E1E10E941736E02934
:1045220011F0E1E07E2EAE81E6E00E945732EFE02C
:104532000E945C32E2E10E941736E02911F0E2E0CB
:104542007E2EAE81E7E00E945732E0E10E945C32AB
:104552000E947E3211F0E3E07E2E0E94472CD39718
:1045620008F453C00E94952C0E949A2CE72D0E94B9
:10457200A12C10F00E94B42CE72D0E94BB2C0E94AB
:104582008332AC91A13008F43FC00E948A320E946B
:10459200DF2C0E94B8374CF40E9483320E9493327F
:1045A2000E94D7350E949D3223C00E94A6320E94EB
:1045B200002DEF930E94A6320E94092DAF91EA23AB
:1045C20079F00E9483320E9493320E94DC35A093DC
:1045D2009403B0939503809396039093970308C036
:1045E2000E94A6320E94122D1CF00E94A8320CC01A
:1045F200A0919403B09195038091960390919703B3
:104602000E942B2D0E94302D04C00E94752C0E9406
:10461200A832AE81AD3029F50E94B730FF93EF93F7
:104622000E94832F0E94BC300E946F30AF91BF91D5
:104632000E94C1303696FF93EF930E94B7320E94D8
:104642006F30AF91BF910E94C1303796FF93EF93C5
:104652000E94B7320E941837AF91BF91EC93E0E20B
:10466200EDA7AE81A53141F4EEE30E94E42FECE028
:104672000E94E92FE0E6EDA70E947B32EEE00E9465
:104682005C32E1E10E941736E029B1F00E94BD32AE
:10469200E4E00E94C13228F00E94B7300E94C73283
:1046A200EC930E94472C1A9728F00E94CA320E946B
:1046B200FC30EC930E94D132AE81E6E00E94573288
:1046C200EFE00E945C32E2E10E941736E029B1F08D
:1046D2000E94BD32E2E00E94C13228F00E94B7304F
:1046E2000E94C732EC930E94472C1A9728F00E942E
:1046F200CA320E94FC30EC930E94D132AE81E7E0D4
:104702000E945732E0E10E945C320E947E32B1F098
:104712000E94BD32E1E00E94C13228F00E94B7300F
:104722000E94C732EC930E94472C1A9728F00E94ED
:10473200CA320E94FC30EC930E94D132AE81A43185
:10474200B1F40E94B7300E94D8320E94EC300E942D
:10475200C13036960E94D8320E94582F0E94FC30F7
:104762000E94C13037960E94D8320E941832AE8120
:10477200A63129F40E947232EBE00E94F131AE813F
:10478200A73129F40E947232E0E40E94F131AE8135
:10479200A83129F40E947232ECE00E94F131AE811C
:1047A200A931E1F4A091E303AA2322F40E94843008
:1047B2000E948C300E94B730BF010E9491300E944B
:1047C200FF2B0E949D300E94DE320E9491300E9497
:1047D2000332DB01EC93E7E70E94EE2FAE81AA31B0
:1047E200B1F40E94B7300E94E4320E94EC300E9481
:1047F200C13036960E94E4320E94582F0E94FC304B
:104802000E94C13037960E94E4320E941832AE8173
:10481200AB3169F4ECE70E947832E8E70E94EE2FB0
:104822000E94F7300E946B320E94FC30EC93AE8102
:10483200AC3149F4E0E30E94E42FEDE60E94E92F57
:10484200E4E50E94EE2FAE81AF3149F4EEE30E941F
:10485200E42FEDE60E94E92FE3E70E94EE2FAE81FE
:10486200A53229F40E94EA32E5E00E94EE2FAE81E1
:10487200A63229F40E94EA32E8E00E94EE2FAE81CD
:10488200A73229F40E94EE32E3E60E94EE2FAE81B7
:10489200A83229F40E94EE32E8E70E94EE2FAE81A0
:1048A200A93249F4E7E70E94E42FE0E40E94E92FED
:1048B200E8E70E94EE2FAE81AB3231F4E9E30E94C9
:1048C200F232EEE00E94EE2FAE81AC3231F4ECE730
:1048D2000E94F232EDE60E94EE2FAE81AD3231F44B
:1048E200E0E00E94F532E0E00E94EE2FAE81EDE1C1
:1048F2000E945732EEE10E941736E02921F1E3E7E8
:104902000E94F131E8E30E94F631AE81AD3111F43B
:10491200EEE501C0E8E7DE01A45BBF4FEC930E9425
:10492200F8321A9748F00E94DE320E94F8320E9452
:10493200582F0E94FC30EC930E94FD32BF010E946E
:10494200F8320E9418320E947B32E6E00E945C320A
:10495200E7E00E941736E02919F0E3E70E94F131FF
:10496200AE81EEE00E945732EFE00E945C32E0E15D
:104972000E941736E02949F0EDE60E94F131E9E79D
:104982000E94F631E4E50E94FB31AE81E1E10E9432
:104992005732E2E10E945C320E947E3219F0E8E76F
:1049A2000E94F631AE81EFE10E942B360E2EE5E237
:1049B2000E942636E02161F0EDE60E94E42FE8E550
:1049C2000E94E92F0E94FD32DF01EE81EF51EC934C
:1049D200AE81AE3231F4E9E30E94E42FE8E30E94B3
:1049E200E92FAE81AF3249F4E8E70E94E42FE5E017
:1049F2000E94E92FE7E70E94EE2FAE81A03331F447
:104A0200E0E30E946F32E0E50E94EE2FAE81A13317
:104A1200B1F4E3E70E94F232E8E70E94EE2FA091A0
:104A22000203A43160F0E4E50E94F131EDE60E9458
:104A3200F631E0E30E94FB31EDE30E943232AE81B7
:104A4200A23341F4EEE30E94E42FEBE00E94E92F4F
:104A5200E0E6EDA70E9461320E943F36E02149F074
:104A6200E0E00E941B32E1E70E942032E1E70E946F
:104A72002532AE81AC3549F4E7E70E94E42FE9E341
:104A82000E94E92FE9E30E94EE2FAE81AD3509F0D5
:104A92008EC0ACA5A83008F044C0E7E70E94F5320A
:104AA2000E94FD32ACA5A083E7EAE0937A000E945F
:104AB200082CE0934603F0934703E7E2E0937A0081
:104AC2000E940233A83EE3E0BE0740F00E943A3162
:104AD200BF010E9402330E94E130EC930E94023334
:104AE200A436E0E0BE0740F00E944731BF010E94B9
:104AF20002330E94EC30EC930E9402331A9750F07A
:104B02000E94F730BF010E9402330E94582F0E9478
:104B1200FC30EC930E945231BF010E9402330E948A
:104B22001832ACA5A830F1F4E6E70E947832E8E347
:104B32000E94EE2F0E944731DF01E0914203E170B3
:104B42000E94C1303E96DF01E0914203E695E1709A
:104B52000E94C1303F96DF01E0914203E695E6955F
:104B6200E170EC93ACA5A93011F5E3E70E94E42FC4
:104B7200E4E70E94E92FE0E30E94EE2F0E940F2F4C
:104B82001A974CF00E944731BF010E940F2F0E94DA
:104B9200FF2B0E949D300E94F730BF010E940F2F11
:104BA2000E940332DB01EC93E7E70E942532AE81DB
:104BB200AE3591F50E94232FA2E8B3E00E94C52AE8
:104BC200A091E303AA2342F4E0918203F0918303CC
:104BD2000E94E1350E948C300E94B730BF010E94D2
:104BE2009130E4E6F0E00E9400320E94DE320E9440
:104BF20091300E94FF2B0E949D300E94FD32BF0126
:104C02000E9491300E940332DB01EC93EEE50E9498
:104C1200F131E1E00E94F631AE81AF3531F4EEE5DB
:104C22000E94F131E2E00E94F631AE81A03631F409
:104C3200E8E30E94F532EDE00E94EE2FAE81A1364C
:104C420031F4E8E70E947832EEE30E94EE2FAE8163
:104C5200A23661F4E8E30E94E42FFE01EF5BFF4F0E
:104C62003696A0913003A083E0E1EDA7AE81A33692
:104C720099F4E8E30E94F5320E949D2EEA17FB07A1
:104C820018F4ECE00E94EE2F0E949D2E0E94A42EAA
:104C920019F0EBE00E94EE2F51E0503108F089C08C
:104CA2000E944F32EC91E03021F40E944F32EFE348
:104CB200EC930E944F32AC91A63021F40E944F3205
:104CC200EDE7EC930E944F32AC91A13021F40E94A7
:104CD2004F32E6E0EC930E944F32AC91A23021F4C5
:104CE2000E944F32EBE5EC930E944F32AC91A3301D
:104CF20021F40E944F32EFE4EC930E944F32AC91C8
:104D0200A43021F40E944F32E6E6EC930E944F3227
:104D1200AC91A53021F40E944F32EDE6EC930E9453
:104D22004F32AC91A73021F40E944F32E7E0EC936E
:104D32000E944F32AC91A83021F40E944F32EFE72B
:104D4200EC930E944F32AC91A93021F40E944F3271
:104D5200EFE6EC930E944F32AC91AA3021F40E940C
:104D62004F32E0E0EC930E944F32AC91AB3021F431
:104D72000E944F32E1E0EC930E944F32AC91AC3092
:104D820021F40E944F32E8E0EC930E944F32AC9142
:104D9200AD3021F40E944F32E0E4EC930E944F3296
:104DA200AC91AE3021F40E944F32E9E0EC935F5FA8
:104DB20074CFE0910103E695E6950E9407330E94C5
:104DC2000D330E9412330E940D330E941A330E9447
:104DD2000D330E9425330E940D330E942A320E9415
:104DE2002C330E942F330E942C330E9434330E94B2
:104DF2002C330E943933E9ABE0910103E695E69545
:104E0200E6950E9407330E943F330E9412330E94AC
:104E12003F330E941A330E943F330E9425330E947F
:104E220044330E942A320E9449330E942F330E9447
:104E320049330E9434330E9449330E943933EAAB2A
:104E4200E0910103E6950E9407330E9444330E94D9
:104E520012330E9444330E941A330E9444330E9448
:104E620025330E943F330E942A320E944C330E9413
:104E72002F330E944C330E9434330E944C330E94E1
:104E82003933EBABFE01E75BFF4FE0810E94073352
:104E92000E944F330E9412330E944F330E941A33F2
:104EA2000E944F330E942533EFA50E942A32EA2B3B
:104EB200AE2FEFA50E942F33EA2BAE2FEFA50E9453
:104EC2003433EA2BAE2FE0910103E170EA2BECAB15
:104ED2000E9454330E9407330E9454330E94593374
:104EE2000E9454330E945F330E9454330E946833FD
:104EF2000E9472330E9476330E9479330E94763385
:104F02000E9480330E947633E295E170EA2BEDAB8A
:104F12000E9487330E9407330E9487330E945933CD
:104F22000E9487330E945F330E9487330E94683356
:104F3200E2950E942A320E948C330E9479330E94A9
:104F42008C330E9480330E948C33E295E170EA2B0D
:104F5200EEABEFA50E9493330E9487330E94123377
:104F62000E9487330E941A330E9487330E9425339E
:104F72000E9497330E942A320E949C330E942F3350
:104F82000E949C330E9434330E949C330E94393326
:104F9200EFAB0E949F330E9407330E949F330E940F
:104FA20059330E949F330E945F330E949F330E94B5
:104FB20068330E94A4330E942A320E949C330E94CA
:104FC20079330E949C330E9480330E949C33E29585
:104FD200E170EA2BE8AF0E94A9330E9407330E94D6
:104FE200A9330E9459330E94A9330E945F330E9461
:104FF200A9330E946833EE1FE0E0EE1F0E942A32BE
:105002000E94AE330E9479330E94AE330E948033F5
:105012000E94AE33E295E170EA2BE9AFEEA5E2958C
:105022000E9407330E94A9330E9412330E94A933BF
:105032000E941A330E94A9330E9425330E944F33E3
:105042000E942A320E94B5330E942F330E94B53348
:105052000E9434330E94B5330E943933EAAF0E9472
:10506200B8330E9407330E94B8330E9459330E941A
:10507200B8330E945F330E94B833E695E695E69511
:105082000E94BD330E2EA0E035FCA1E0EA2FEE0F08
:10509200EE0FEE0FE0290E94C233E2950E94C83360
:1050A2000E94C2330E948033EA2B0E94C233E295EF
:1050B200EF70E695E170EA2BEBAFFE01EE5BFF4F7E
:1050C200E081E695E695E6950E940733FE01EE5BE8
:1050D200FF4FE081E695E6950E94CD330E94C233F0
:1050E2000E94D1330E94C2330E94BD33AE2FEEA57F
:1050F2000E947233EA2BAE2FEEA50E94D833AE2F58
:10510200EEA50E94DB33EEA5E695E170EA2BECAF4B
:10511200EEA50E9493330E94E033E2950E94CD33C4
:10512200AE2F0E94E0330E941A330E94E0330E94A5
:10513200E533AE2F0E94E0330E947233EA2BAE2F8A
:105142000E94E0330E94D833AE2F0E94E033E695EE
:105152000E94DB330E94E033E170EA2BEDAFEEA553
:105162000E94A4330E940733EDA50E94CD33AE2FD7
:10517200EDA50E94D133AE2FEDA5E695E6950E94EE
:10518200BD33AE2FE0910103E2950E942A32EA2B51
:10519200AE2FEEA5EE1FE0E0EE1F0E94C833AE2F49
:1051A200EDA5E695E695E6950E94DB33EDA5E29541
:1051B200E170EA2BEEAFEDA50E9493330E94E93332
:1051C200E2950E94CD33AE2F0E94E9330E941A333A
:1051D2000E94E9330E94E5330E94EE330E9472334B
:1051E200EA2B0E94EE330E94D8330E94EE33E695FA
:1051F2000E94DB330E94F433E170EA2BEFAFFE0131
:10520200F09670960F01EDA50E94A4330E94073319
:105212000E94F433E2950E94CD330E94EE330E9445
:105222001A330E94F4330E94E533AE2F0E94E93311
:105232000E947233EA2BAE2F0E94E9330E94D833C8
:10524200AE2F0E94E933E6950E94DB330E94E933D8
:10525200E170EA2BD001EC9333FE0DC051E05131E5
:1052620050F4E52FF0E0DE01D096AE0FBF1FEFEF56
:10527200EC935F5FF4CF0E94F9335D3078F40E94C3
:10528200FF33A2E5B8E00E94F535E17011F45D98B4
:1052920001C05D9A0E9406345F5FEFCF0E940E3418
:1052A2005D3078F40E94FF33A0E3B8E00E94F53548
:1052B200E17011F45D9801C05D9A0E9406345F5F4F
:1052C200EFCF0E940E345D3078F40E94FF33A2E0EB
:1052D200B8E00E94F535E17011F45D9801C05D9A65
:1052E2000E9406345F5FEFCF0E940E345D3078F487
:1052F2000E94FF33A6E0B8E00E94F535E17011F498
:105302005D9801C05D9A0E9406345F5FEFCF0E94F4
:105312000E345A3098F45E9885E28A95F1F7E9E006
:10532200E51BA0E4B1E00E94F535E17011F45D984F
:1053320001C05D9A0E9406345F5FEBCF41E04131CC
:10534200E8F451E05930C0F45E9885E28A95F1F7AD
:10535200E42FF0E0DE01D096AE0FBF1FAC91E8E083
:10536200E51B0E94ED35E17011F45D9801C05D9A74
:105372000E9406345F5FE6CF4F5FE1CF5D9A85E220
:105382008A95F1F7289A8DEC9AE00197F1F70E943D
:10539200372DA92DEAE00E9435360E2AAB2DEAE020
:1053A2000E9435360E2AAA2DEAE00E943536E029FF
:1053B20029F0E0E0E0936003E0936103A82DE4E6C6
:1053C2000E943A360E2EA0E0F099A1E00E94692DCB
:1053D20029F00E94752BF09AE89433F80C94130686
:1053E200FFCFAA93E091C000E072E1F3E881E0937D
:1053F200C60021960895A0914A03B0914B030895E7
:10540200A091B403B091B5038091B6039091B70314
:105412000895E0E0F0E061EE75E40E9466350895DB
:10542200E0915603F09157030895662777270E946B
:105432008E340E944D370895E0916203F091630328
:105442000895A091BC03B091BD038091BE039091D9
:10545200BF030895E0E0F0E060E271E40895A091F6
:105462005603B09157030895E0E0F0E00E946336DE
:105472000895A0916203B09163030895E091E4035B
:10548200F091E5036091E6037091E70308950E94AD
:105492005534ED93FC930895A091D003B091D103BC
:1054A2008091D2039091D303E0E0F0E06AE774E4E4
:1054B2000E941835DF01CB01ACCFA091CC03B09193
:1054C200CD038091CE039091CF030895A091F00374
:1054D200B091F1038091F2039091F3030895E0916A
:1054E2006E03F0916F0360917003709171030895E0
:1054F200A4E6B0E080E090E00E949136DF01CB01AB
:10550200E091CC03F091CD036091CE037091CF0373
:105512000E945C3708950E9461370E94C134089549
:10552200E0916803F09169030895E0936803F093B2
:1055320069030895A091EC03B091ED038091EE030D
:105542009091EF030895E093EC03F093ED036093E1
:10555200EE037093EF030895A0916E03B0916F0371
:10556200809170039091710308950E949136DF013A
:10557200CB01E091EC03F091ED036091EE037091A9
:10558200EF030E945C37C7CF0E945734ED93FC9320
:105592000895E0E0F0E061EE75E40E9418350895A8
:1055A200A091D403B091D5038091D6039091D703F3
:1055B2000895E0E0F0EC69E774EC0E94AB350895E1
:1055C200E7EEF3E0E0938403F09385030895E0911E
:1055D200D403F091D5036091D6037091D703089557
:1055E200E091D803F091D9036091DA037091DB0363
:1055F2000895A091B803B091B9038091BA03909134
:10560200BB030895E093B803F093B9036093BA0320
:105612007093BB030895A091C003B091C103809120
:10562200C2039091C3030895E091B803F091B903C6
:105632006091BA037091BB030895A091C803B09121
:10564200C9038091CA039091CB030895E0916A0344
:10565200F0916B0360916C0370916D030895E09378
:105662006A03F0936B0360936C0370936D03089568
:10567200EDDFAAE4B0E00E9482370895A0916A03A8
:10568200B0916B0380916C0390916D030895E0E0FB
:10569200F0E060E070E00895DDDE0E9418350895C4
:1056A200E0E00E943A360E2E0895A0919803B09140
:1056B200990380919A0390919B0308950E22A091E1
:1056C2002503ECE30E9435360895A0916003B09162
:1056D20061030895A0915E03B0915F03C5CEE0918E
:1056E2005E03F0915F030895A4E6B0E00C941834D1
:1056F200E7EAE0937A00A4E00C94AD03EF2FF0E028
:105702006E2EE7E2E0937A000895E7EAE0937A00EA
:10571200A3E00E94AD03EF2FF0E09E2EE7E2E093BC
:105722007A000895E7EAE0937A00A1E00E94AD03CF
:10573200EF2FF0E0BE2EE7E2E0937A000895E0E07A
:10574200F0E00E948A370895EBE0E093F903E8EB7A
:10575200E093FA030895E8ECF0E0E0937403F09329
:1057620075030895E0EDF7E0E0937603F093770395
:105772000895E0934E03F0934F0308950E940D366F
:105782000E948E340E944D370895E0935403F093A3
:1057920055030895E0936E03F0936F0360937003D3
:1057A200709371030895E0935E03F0935F0308958D
:1057B200E0936403F09365030895E0938803F09304
:1057C20089030895E0E0E0930D04E0930203089555
:1057D200E0E0E093F403E093F503E093F603E09353
:1057E200F703E093F8030895E0E0E093FB03E0930E
:1057F200FC03E093FD03E093FE030895EAE0F0E08A
:105802000E94D4360895AAE0B0E00C9418340E94A5
:10581200AD030E9402360E94FE350895E7EAE09346
:105822007A00A0E00E94AD03EF2FF0E00895E0932C
:105832009C03F0939D0360939E0370939F030895CE
:10584200E0914E03F0914F030895E0919C03F09193
:105852009D0360919E0370919F030895E7E2E09398
:105862007A008AE48A95F1F708958AE48A95F1F735
:10587200E7EAE0937A000895A7E00E94AD03EF2FD4
:10588200F0E0E0934403F09345030895A0914403AC
:10589200B09145030895A12FE2E30E943A360E2EFD
:1058A20008950E2EA52DE1E00E943A360E22AE8D0D
:1058B200E0E00E941736E02108950E2EA52DE1E0CA
:1058C2000E943A360E22AD8DE0E00E941736E021AA
:1058D2000895E4E00E943536E0210895F0E0E09377
:1058E2004403F09345030895E0E0E0934403E0931A
:1058F20045030895E4E00E9417360E2E0895AD8DFB
:10590200E5E00E9417360895AA2DEAE00E94353696
:105912000E2E0895A0E0F3FCA1E0E0E00E9417360D
:105922000E22A22FE3E60895E0914403F09145038D
:105932000895F297ADE7B0E00E9489360F0108950D
:10594200F0E0DE019396AE0FBF1FEC91F0E0D001C4
:105952000E94C136E0934403F093450397DFA93CCC
:10596200E0E0BE070895E8ECF0E0E0934403F09332
:1059720045030895F0E0DE019796AE0FBF1FEC914C
:10598200F0E084DF0E948936DF01E4E6F0E00E9465
:10599200C136E0934403F09345030895E02FF0E00D
:1059A200DE015F96AE0FBF1F0895A0919003B091E4
:1059B200910380919203909193030895E8EEF3E0AE
:1059C20060E070E00E94FE36DF01CB01ADDF6627AA
:1059D20077270895EC91F0E0A0E4BCE90E94C1367B
:1059E200E4DF662777270895E0939003F09391030D
:1059F20060939203709393030895D7DFDFCF0E94E1
:105A0200DC35E5E0F0E060E070E00E948136089568
:105A12000E94DC35E4E1F0E060E070E00E9479365B
:105A220008950E94DC35A431E0E0BE07E0E08E0775
:105A3200E0E09E070895E0919803F0919903609148
:105A42009A0370919B03A0E5B4E180E090E00E948C
:105A5200BC36CACFE8EEF3E060E070E008950E9441
:105A6200FE36E0934403F09345030895A62DEAE041
:105A72000E9435360E2E0895A22FE3E60E94353697
:105A82000895A0E0F0FCA1E0E0E00E941736E021DA
:105A92000895FCDEE0E0F0E00E943F360895E894CD
:105AA20025F8E0E0E09327030895F0DEDDCC0E2236
:105AB200A0E022FCA1E0E1E00E941736E021089577
:105AC200E0933403ECCFE0E00E9417360E220895F3
:105AD200E0E00E941736E0210895E0E00E941736C8
:105AE2000E2E0895E0910403F0E03597CFDE0E9478
:105AF2005D360E2EE0913303D8DDFF276627772728
:105B02000895E1E00E9417360E2E0895A0E022FCCF
:105B1200A1E0DECFE989FA89A0919C03B0919D03AF
:105B220080919E0390919F03662777270E94793682
:105B32000E2EEAE0F0E060E070E00E948136089507
:105B4200E0937403F093750308957FDEA989BA89FF
:105B5200882799270E94DC350895A630E0E0BE0729
:105B6200E0E08E07E0E09E070895A0917403B091F3
:105B720075030895E0917403F09175030895E9891E
:105B8200FA89A0919C03B0919D0380919E0390910C
:105B92009F03662777270895E0934403F093450314
:105BA2000895E32FA091E003B091E1038091E20315
:105BB2009091E303FF27662777270E948E3408958A
:105BC20065DEEAE00E94B1360895E32FF0E0A0918D
:105BD200E003B091E1038091E2039091E3030E941C
:105BE2000D360E948E3497CCA0917603B091770344
:105BF20008950E9412360E945E378DCCA32FBB27D8
:105C0200E091E003F091E1036091E2037091E3031C
:105C1200F0CFE0917603F091770308950E940D365C
:105C22000E948E340895E09116033FDDFF27662718
:105C320077270895E0937E03F0937F030895E09120
:105C42001603F0E032DD0E940D360E94DC35089525
:105C52000E94B736A0917E03B0917F030895E09130
:105C62007E03F0917F030895A0911603BB27E09174
:105C72009803F091990360919A0370919B030E949B
:105C820012360E94DC350895E1E00E941736E021C9
:105C92000895A0E0F099A1E0E1E00E9417360ECD50
:105CA2000E22A22FE3E60E941736E02108950E2E5F
:105CB200A0912503ECE30E9435360E2208950E943E
:105CC2008A37A1E0B0E00C941834E091CC03F09153
:105CD200CD036091CE037091CF03AAE3B0E00E949E
:105CE2005734EDCFA2E4B0E00E945734E8CF18DC7D
:105CF200A4E4B0E0E4CF0E949237A1E0B0E00C94BB
:105D02001834EAE00E943A360E2E0895AB2DEAE0EE
:105D12000E9435360E2EA0E027FCA1E0D4CEA09141
:105D22003003E3E00E9417360E2E0895E09130030F
:105D3200F0E0E25EFC4F0895EB85FC850E9402369E
:105D4200A62DB0E008950E9457360E2EA62DEAE049
:105D52000E943A36E0210895A92DEAE00E943536E4
:105D62000E2E0895E0910D03F0E0E85FFC4F0895D8
:105D7200E0915403F09155030895A22FE3E60E94A7
:105D82001736E0210895E0913903EF5FE09339037C
:105D9200E0913803A0913903EA1708950E9435363D
:105DA2000E2EA0E023FCA1E00895A0915403B0912F
:105DB20055030895A0916803B09169030895A091D5
:105DC2003003B0E0A25EBC4FEC910895AE81E3E6F1
:105DD2000E9417360E2EB0CFE1E00E946A37EA1B0E
:105DE2000E94BD370895A091E003B091E103809134
:105DF200E2039091E3030895E091E003F091E1035F
:105E02006091E2037091E3030895E093E003F0935D
:105E1200E1036093E2037093E3030895A0918E037C
:105E2200B0918F030895E8DFA0E0B0E080E09FE347
:105E32000895E093D003F093D1036093D20370935B
:105E4200D3030895D0DF28CCD7DFA2E8B3E09CCB00
:105E5200EA1BFB0BE3DEDF01CB01EAE9F9E969E2C8
:105E620071E40E946635DF01CB01E0E0F0E068E515
:105E720071E451CBA6E8B3E087CBEE0FFF1FA0E0A1
:105E8200B4E00E946737E4CFE2E0F0E00E94D4364B
:105E92000895E0938603F09387030895E091B00399
:105EA200F091B1036091B2037091B3030895EAE0F7
:105EB200F0E00E94C1360895A091B003B091B10301
:105EC2008091B2039091B303089509DB11CBE09363
:105ED200AC03F093AD036093AE037093AF030895E8
:105EE200E0E00E943A36E0210895ED85FE85A0911A
:105EF2009C03B0919D0380919E0390919F0366271E
:105F020077270895A0919C03B0919D0380919E03F1
:105F120090919F030895BADCAE0FBF1FE12FF0E00E
:105F2200EA0FFB1FE0935203F093530308950E947C
:105F3200F229A0E00C94F2290E94F229E091530385
:105F4200AE2F0E94F229A09152030C94F229F0E0A4
:105F5200AE0FBF1FE0911903F0E00895F0E0AE0F1D
:105F6200BF1FE0913C03F0E0AE0FBF1FE0913D0385
:105F72000895F0E0EA0FFB1FE0935203F0935303FE
:105F820008950E94F229A09114030E94F229A0917F
:105F920015030C94F2290E94F229A09119030C9482
:105FA200F229A0E00E94F229A09152030C94F22956
:105FB200DE01AE5BBF4FEC930895EAE0DE01AC5B1D
:105FC200BF4FEC930895DE01AA5BBF4FEC93089597
:105FD200DE01A95BBF4FEC930895DE01A85BBF4FC2
:105FE200EC930895EAE0DE01A75BBF4FEC93DE017C
:105FF200A65BBF4FEC93DE01A55BBF4FEC93DE01C6
:10600200A45BBF4FEC93DE01A35BBF4FEC93DE01B9
:10601200A25BBF4FEC93DE01A15BBF4FEC93DE01AD
:10602200A05BBF4FEC930895E9E0EFA7E091360340
:10603200E170EE0FAE2FE0913603E695E170EE0FC0
:10604200EE0FEE0FEA0F0E2E0895E0913603E6955D
:10605200E695E170AE2FE0E0F5FCE1E0EA2BEE0F11
:10606200EE0FE00DEEA70895EFA7E0913603E17081
:10607200EE0FAE2FE0913603E695E170EE0FEE0FD4
:10608200EE0FEA0F0E2EE1CFE295E07FEE0FEE0F5C
:106092000895E0E020FCE1E0E0930103A091A00379
:1060A200B091A1038091A2039091A3030895A091BE
:1060B200A003B091A1038091A2039091A30308953C
:1060C200AA30E0E0BE07E0E08E07E0E09E07089518
:1060D200ECDAEAE0F0E060E070E008950E94FE365B
:1060E200DF01CB01EAE0F0E060E070E00E941837E7
:1060F2000895FE01EF5BFF4F34960895DE01AC5B1D
:10610200BF4FEC930895E0918003F09181030E94C8
:10611200E135DF0173CBE0938203F09383030895AB
:10612200A0918203B09183030895FE01EF5BFF4FBC
:106132003196BF01F5DF62CBDF01EAE0F0E00E94B9
:106142000637DB01EC930895FE01EF5BFF4F3296B9
:10615200BF01E6DFEAE0F0E00E940637DB01EC93E4
:106162000895A0918603B09187030895FE01EF5B25
:10617200FF4F35960895E4E6F0E060E070E00895A0
:10618200EC93FE01EF5BFF4F089591DFEAE0F0E050
:1061920060E070E00895A0E020FCA1E0EA2FE29523
:1061A200E07FAEA5EA0FEEA70895A0914C03B0914F
:1061B2004D030895FE01EF5BFF4F3D96BF01F5CF02
:1061C200E8EEF3E00E94C136DF01EAE0F0E00E946F
:1061D2000337DB010895E4E6F0E00E94C136DF01F7
:1061E200EAE0F0E00E940337DB010895FE01EF5B75
:1061F200FF4F3E960895DF01EAE0F0E00E94033788
:10620200DB0108950E940337DB01EC930895E2E07D
:10621200DE01A75BBF4FEC930895BB27EAE0F0E0F5
:106222000E940637DB010895FE01EF5BFF4F3B96AC
:106232000895FE01EF5BFF4F3A9608950E94D9360A
:10624200DF01CB01EAE0F0E060E070E00E94143789
:106252000895A031E7E2BE07E0E08E07E0E09E0786
:106262000895A83EE3E0BE07E0E08E07E0E09E0767
:106272000895FE01EF5BFF4F3C960895A436E0E0DF
:10628200BE07E0E08E07E0E09E070895FE01EF5BA7
:10629200FF4F3D960895F2D9EAE0F0E060E070E049
:1062A2000895FE01EF5BFF4F3F960895DE01A65B66
:1062B200BF4FEC93E4E7DE01A55BBF4FEC9308957B
:1062C200E0E4DE01A15BBF4FEC930895DF01CB0157
:1062D200E0E0F0E060E171EC0E94AB350895E0E4AB
:1062E200DE01A25BBF4FEC930895DF01CB01E0E03A
:1062F200F0E066EC72EC0E94AB350895E0E4DE015A
:10630200A35BBF4FEC930895DF01CB0152C9E0E4D8
:10631200DE01A45BBF4FEC930895A091A403B0915A
:10632200A5038091A6039091A7030895F6DFEAE002
:10633200F0E060E070E00895EFA5E058EFA7EEE32B
:10634200B5CFE0917C03F0917D030E94E135E093AB
:106352007C03F0937D030895C2D8A4E6B0E080E008
:1063620090E003C9A0917C03B0917D030895BF0121
:10637200F9DFE0E1F7E20E94D436DECEBF01F2DFC0
:10638200E8EEF3E00E94D436D7CEBF01EBDFE4E6BD
:10639200F0E00E94D436D0CEBF01E4DFEAE0F0E0C4
:1063A2000E940637DB01EC930895E0E5DE01A45B71
:1063B200BF4FEC930895A0918403B0918503089593
:1063C200BF01F9DFE4E6F0E00E94D436B5CEBF01AA
:1063D200F2DFEAE0F0E00E940637DB01EC93089579
:1063E200DE01A65BBF4FEC930895DE01A55BBF4FB4
:1063F200EC930895DE01A45BBF4FEC9308950E94D5
:10640200D4369ACEEAE0F0E00E9406370895A12F32
:10641200B0E03ACDEF85F889F695E79508950E94A8
:10642200C136E9CEA0915803B09159030895EAE02C
:10643200F0E0E8CEDE01A25BBF4FEC930895DE01EF
:10644200A15BBF4FEC930895DE01A05BBF4FEC93BD
:106452000895E170EE0FEE0FEE0F0895ECE7C5DF41
:10646200A4CFDE01A35BBF4FEC930895AD8DE4E0B2
:106472000E941736AE2FE0E020FCE1E0EA23089507
:10648200AE2FE0E020FCE1E0EA230895ECE7D2DF62
:10649200E0E5D5CFE7E7CEDFE9E3D1CFE52FF0E0C6
:1064A200DE01AF5BBF4FAE0FBF1F08950E941736CC
:1064B2000E2EAE8108950E9417360E2AAE810895DF
:1064C200AE81E2E30E9417360E2EAB89BC89E4EA64
:1064D200F1E00895BF01AB89BC89E9CC74DDE9E73D
:1064E20077CDE9E370DDE0E573DDEEE376CD6BDDDC
:1064F200E7E76ECDAE81E5E0D9CFE3E10E94173642
:10650200E0290895E72DF0E0DE015F96AE0FBF1F90
:106512000895A0919403B091950380919603909170
:1065220097030895EC91F0E0A0E4BCE90E94C13623
:10653200F0DF662777270895E0939403F09395039D
:1065420060939603709397030895E3DF37CAE0914F
:106552009803F091990360919A0370919B03A0E5CF
:10656200B4E180E090E00E94BC36E6CFCBDCEAE00A
:10657200F0E060E070E00895D7D9F695E7950CCB8E
:10658200EDA784D9A436E0E0BE070895BF017ED905
:1065920022CEFE01EF5BFF4F3696BF0177D987CC43
:1065A200FE01EF5BFF4F3796BF0170D940CFBF01AD
:1065B200A0916603B09167030895FE01EF5BFF4F60
:1065C2003696BF010895BF01A0915003B0915103C7
:1065D2000895E8E5F8DCE4E5FBCCEDE6F4DCE8E37D
:1065E200F7CCF1DCE0E5F4CCEEDCEEE5F1CCA09109
:1065F2005C03B0915D030895FE01EF5BFF4F379698
:106602000895A0914603B09147030895E170E7957C
:10661200E0E0E795AE2F0895FE01EA5BFF4FE081CF
:106622000895E295EF70E695E1702EDDEA2BAE2F2C
:106632000895E295EF70E695E695E170E295E07FC8
:10664200EE0FEA2BAE2F0895E295E170E295E07F1E
:10665200EA2BAE2F0895EA2BAE2FDECFE695E1703E
:10666200EE0FEE0F0895E695E695E170EE0F0895B0
:10667200E695E695E695E170EA2B0895FE01E95B61
:10668200FF4FE0810895FE01E85BFF4FE08108952E
:10669200EA2BAE2FF8CFEA2BAE2FF0CFFE01E65B4E
:1066A200FF4FE0810895FE01E25BFF4FE081089514
:1066B200E695E170E9DCEA2BAE2F0895E695E695C2
:1066C200E170E295E07FEE0FEA2BAE2F0895E6959A
:1066D200E695E695E170E295E07FEA2BAE2FEFA515
:1066E2000895E695E695E695B4CEEA2BAE2FDBCF7C
:1066F200E295EF70E695E170EE0FEE0F0895E295E8
:10670200EF70E695E695E170EE0F0895FE01E35B0A
:10671200FF4FE0810895EA2BAE2FFE01E15BFF4FB0
:10672200E0810895E295EF70E69570CFFE01E45B9B
:10673200FF4FE0810895EA2BAE2FF8CFFE01E15B17
:10674200FF4FE0810895E295EF70E695E695089592
:10675200FE01E55BFF4FE0810895EA2BAE2FFE01BB
:10676200E05BFF4FE0810895EA2BAE2F97CFFE0149
:10677200E05BFF4FE0810895E170E295E07FEA2B54
:106782000895AE2FFE01EE5BFF4FE0810895E170A8
:10679200EE0FEE0FEA2B0895E17076DCEA2B0895F6
:1067A200E695E170E295E07FEE0FEA2B0895E6951B
:1067B200E695EDCFE170EE0FEA2BAE2F0895FE01C4
:1067C200ED5BFF4FE0810895E295EF70E695D4CF3F
:1067D200FE01EC5BFF4FE0810895AE2FFE01EB5B03
:1067E200FF4FE0810895FE01EB5BFF4FE0810895CA
:1067F200289885E28A95F1F751E008955E9885E23E
:106802008A95F1F7ECE0E51B089585E28A95F1F7A8
:106812005E9A85E28A95F1F708955D9A85E28A95F6
:10682200F1F7289A84E191E00197F1F7E1CF109610
:1068320039F08DEC9AE00197F1F7A8951197C9F715
:10684200089530976040704009F0705808955523BC
:1068520042F4503811F4E0FF04C03196691F791FE9
:106862006BF050E8572711F45F93CFC05F3F31F0D0
:10687200660F000C57956795752F08955F9300205A
:106882000AF0CFC0C8C050E8192E1522880F991FF0
:106892009527550F879550E8072E0522660F771F1B
:1068A2007527550F67950895689401C0E8945F9322
:1068B200F2DF703818F07F3F08F4A7C056E1571B8B
:1068C200AAF4519558300EF4593030F0EFEFFFEF43
:1068D2006FEF7FE777F91AC077275523B9F0EE0FEC
:1068E200FF1F661F771F5A95D1F710C077275830C0
:1068F20028F0EF2FF62F672F5850F9CF552331F09C
:1069020076956795F795E7955A95D1F700200AF4A1
:106912005BD15F910895689401C0E894309760401C
:106922007040B1F0002426F0772312F400944CD189
:10693200172E7EE1112032F07A95EE0FFF1F661FAF
:10694200111CF9CFEF2FF62F612D5F938ADF5F9134
:1069520008954F93AF01FD01DA01AB01BC01CA01F9
:10696200402D012C142E4F910895EA0FFB1F681F32
:106972000895E095F0956095EF5FFF4F6F4F089592
:106982005F9381DF903871F150E8152604C05F9360
:106992007ADF903839F1703821F1572F591B2BF1DA
:1069A20012F4D7DFFACF583118F0AA27BB2788276D
:1069B200583028F0AB2FB82F88275850F9CF5523DD
:1069C20029F08695B795A7955A95D9F7502D512557
:1069D20072F0CBDF38F46795F795E795739513F46A
:1069E20020C0B7DF3EDF5F910895D8F7FBCFEA1BE7
:1069F200FB0B680B51F010F40094BBDF662392F39B
:106A0200EE0FFF1F661F7A95CBF7EE27FF2766274B
:106A120077275F910895EFEFFFEF6FE77FEF5F91C9
:106A22000895EFEFFFEF6FE77FE75F9108955F93C0
:106A32002ADF703851F3903841F301240894791F0A
:106A420023F41CF300203AF3ECCF0F921F932F9301
:106A52003F934F93112722279927689FA0018F9F69
:106A6200302D410D591F6B9F300D411D591F8E9FB7
:106A720027D0BF9F25D06A9F23D0BE9F1DD0AF9F36
:106A82001BD0AE9F110D291F391F491F591FE32F1C
:106A9200F42F652F522F4F913F912F911F910F90FD
:106AA20066232AF0550FEE1FFF1F661F02C0739563
:106AB2004BF2CDDE5F910895100D211D391F02C0EA
:106AC200200D311D491F591F08955F93DCDE703878
:106AD20021F411200AF49FCFA4CF903809F495CF66
:106AE20001240894970B1BF4D4F30020F3CF792FE1
:106AF2001F932F933F934F9311241127222733275C
:106B02004427552790E2AE17BF078607410730F0AA
:106B1200AE1BBF0B860B410B089401C08894551F16
:106B2200221F331F111CAA1FBB1F881F441F9A95C7
:106B320051F7F901612D4F913F912F911F916623DA
:106B420032F0550FEE1FFF1F661F7A9543F27FDE6C
:106B52005F91089599239AF0772342F0971748F0AE
:106B620029F4AE17BF07860720F031F09894889475
:106B72000895989408940895189488940895772312
:106B8200C2F7971798F3A9F7EA17FB07680788F384
:106B920099F3ECCFDFDFE1E009F008F0EE2708958A
:106BA200D9DFE1E009F008F4EE270895EA0FFB1FB0
:106BB200681F791F0895AE1BBF0B860B970B0895B4
:106BC200F195E195F0400895F09560957095E19505
:106BD200FF4F6F4F7F4F0895EE230E2EEA2F19F0CD
:106BE200E6950A94E9F70895EE230E2EFD0121F0B1
:106BF200F695E7950A94E1F70895F695E795F695E7
:106C0200E795F695E795F695E7950895FE2FFF0F20
:106C1200FF0B6F2F7F2F08956F2F660F660B762F56
:106C220008958B2F880F880B982F0895EA17E1E0BB
:106C320009F0EE270895EA17E1E009F4EE27089536
:106C4200AE17E1E00CF4EE270895AE17E1E00CF088
:106C5200EE270895EA17E1E00CF0EE270895AE174B
:106C6200E1E008F4EE270895AE17E1E008F0EE2720
:106C72000895EA17E1E008F0EE270895EA17FB0706
:106C8200E1E009F0EE270895EA17FB07E1E009F4D5
:106C9200EE270895AE17BF07E1E00CF0EE27089546
:106CA200EA17FB07E1E00CF0EE270895EA17FB076D
:106CB200E1E008F4EE270895AE17BF07E1E008F01F
:106CC200EE270895EA17FB07E1E008F0EE270895A2
:106CD200EA17FB0768077907E1E009F0EE27089554
:106CE200EA17FB0768077907E1E00CF4EE2708953D
:106CF200AE17BF0786079707E1E00CF0EE2708956D
:106D0200EA17FB0768077907E1E00CF0EE27089520
:106D1200FA9FF02DEB9FF00DEA9FE02DF10D089503
:106D22007A9F702D6B9F700DF89F700DE99F700D0B
:106D32006A9F602D710DFB9F600D711DE89F600DB4
:106D4200711D8827FA9FF02D610D781FEB9FF00DC2
:106D5200611D781FEA9FE02DF10D681F781F0895CD
:106D62006E2F6A9FF0016B9FF00D089574D0D0DFF3
:106D72000EF426DF08957DD0D3DF0EF425DF0895CB
:106D82000024112490E1AA0FBB1F001C111C0E1A33
:106D92001F0A18F40E0E1F1E01C0A1609A9599F7E2
:106DA200FD01D001089557D0EBDF0EF409DF0895FD
:106DB2003F934F935F93002411244427552730E2D9
:106DC200AA0FBB1F881F991F001C111C441F551FAF
:106DD2000E1A1F0A460B570B28F40E0E1F1E461FD3
:106DE200571F01C0A1603A9559F7FD01BC01D001BE
:106DF200CA015F914F913F9108953BD0D9DF0EF4C4
:106E0200E3DE0895BDDFFD010895E894B7FF04C0F5
:106E1200A095B09511966894F7FDD2DEB1DFFD0121
:106E22000EF4CEDE0895C4DFFD01BC010895E8949E
:106E320097FF09C0A095B09580959095AF5FBF4F21
:106E42008F4F9F4F689477FDBFDEB2DFFD01BC011B
:106E52000EF4BADE0895E894F7FF02C0B1DE68943A
:106E6200B7FF06C0A095B095119600F8039400FAFA
:106E72000895E89477FF02C0A7DE689497FF0BC0DD
:106E82000024A095B095809590951196801D901D37
:106E920000F8039400FA0895ED93FD936D937C93AB
:106EA2000895A881B9818A819B810895E883F98335
:106EB2006A837B830895689401C0E89401D02EDD33
:106EC200182E862F612D192E972F712D1B2EBF2F55
:106ED200F12D1A2EAE2FE12D0895129602D0BF0188
:106EE2001297119602D0FE2F1197F999FECFFF93B8
:106EF200FFB7F894A1BDB2BDF89AE0B5FFBFFF910C
:106F0200089507D012960F01FB0103D0F0011297EA
:106F1200089507D01196EF93EF2F03D0EF911197B9
:106F22000895F99B02C0A895FCCF9FB7F894A1BD24
:106F3200B2BDF89A80B5E81719F0E0BDFA9AF99A4D
:106F42009FBF089500240E160F0606060706089531
:106F520000240A160B06089500240A160B060806DA
:106F620009060895EA17FB07680779070895AE171F
:106F7200BF07860797070895E894EE2309F06894FF
:106F82000895AC0FBD1F05900D928A95E1F7089503
:00000001FF
